S02B00002F686F6D652F766F6F72627572672F446576656C6F706D656E742F4F70656E424C542F5461726765E0
S315080000000000022091650008E1650008E165000826
S31508000010E1650008E1650008E165000800000000E8
S31508000020000000000000000000000000E165000874
S31508000030E165000800000000E1650008E1650008C8
S31508000040E1650008E1650008E1650008E16500086A
S31508000050E1650008E1650008E1650008E16500085A
S31508000060E1650008E1650008E1650008E16500084A
S31508000070E1650008E1650008E1650008E16500083A
S31508000080E1650008E1650008E1650008E16500082A
S31508000090E1650008E1650008E1650008E16500081A
S315080000A0E1650008E1650008E1650008E16500080A
S315080000B0E1650008E1650008E1650008E1650008FA
S315080000C0E1650008E1650008E1650008E1650008EA
S315080000D0E1650008E1650008E1650008E1650008DA
S315080000E0E1650008E1650008E1650008E1650008CA
S315080000F0E1650008E1650008E1650008E1650008BA
S31508000100E1650008E1650008E1650008E1650008A9
S31508000110E1650008E1650008E1650008E165000899
S31508000120E1650008E1650008E1650008E165000889
S31508000130E1650008E1650008E1650008E165000879
S31508000140E1650008E1650008E1650008E165000869
S31508000150E1650008E1650008E1650008E165000859
S31508000160E1650008E1650008E1650008E165000849
S31508000170E1650008E1650008E1650008E165000839
S30D08000180E1650008E1650008CD
S3150800018810B5054C237833B9044B13B10448AFF3BB
S3150800019800800123237010BDB4020020000000006F
S315080001A81C69000808B5034B1BB103490348AFF39C
S315080001B8008008BD00000000B80200201C6900087D
S315080001C872B6704762B67047F0B5002401E001348C
S315080001D8E4B2112C20D8114D15F8147005EB440516
S315080001E895F801E007EB0E0505FB00054AF2104CE9
S315080001F89CFBF5F605FB16C6002EE8D19CFBF5F523
S31508000208ADB20D80013DADB2B5F5806FDFD217707E
S3150800021883F800E00120F0BD0020F0BD5C69000805
S3150800022800B583B001AB0DF105020DF106014FF4D7
S31508000238FA70FFF7C9FF012803D0EE21384800F005
S31508000248D9FD384B00225A611A6842F400421A60EE
S3150800025801E000F0B3FE334B1B6813F4004FF8D1E6
S31508000268304B1A6822F002021A601A6842F0010234
S315080002781A6001E000F0A2FE2A4B5B6813F0010F32
S31508000288F8D09DF805305A1E9DF80430013B1B0529
S3150800029843EA0243BDF80620013A1343214AD361CB
S315080002A8136823F00103136001E000F087FE1D4B75
S315080002B85B6813F0010FF8D11A4BD3F8002242F005
S315080002C80102C3F80022D3F81C2222F00102C3F85F
S315080002D81C22D3F80C2242F00102C3F80C22002291
S315080002E8C3F84022C3F84422D3F8042222F00102B4
S315080002F8C3F80422D3F8142222F00102C3F8142200
S31508000308D3F81C2242F00102C3F81C22D3F80022B3
S3150800031822F00102C3F8002203B05DF804FB00BF0F
S31508000328346900080064004038B504460D46214B78
S315080003389B6813F0806F2FD01E4BD3F8802102F0EC
S315080003480102C3F88021D3F8802142F07C4242F4A6
S315080003580012C3F88021C3F88451E178A278120400
S3150800036842EA0162617842EA012221780A43C3F81F
S315080003788821E179A279120442EA0162617942EA9E
S31508000388012221790A43C3F88C21D3F8802142F047
S315080003980102C3F8802107E04FF4A271064800F06D
S315080003A829FDC9E700F00AFE024B9B6813F0806F27
S315080003B8F8D038BD0064004034690008214BDB6872
S315080003C813F0030F3CD01F4BD3F8B03113F0040FCA
S315080003D80ED11C4BD3F8B0315B0D40F267629342DD
S315080003E80DD00020174AD36843F02003D36070471E
S315080003F8144BD3F8B031DB0843F00043EDE7114B53
S31508000408D3F8B8210270D3F8B821120A4270D3F883
S31508000418B821120C8270D3F8B821120EC270D3F81C
S31508000428BC210271D3F8BC21120A4271D3F8BC2147
S31508000438120C8271D3F8BC311B0EC3710120D1E7A7
S31508000448002070470064004008B5FFF7B9FE08BDEC
S3150800045810B500F003FA00B910BD03F081FA0028B8
S31508000468FAD000F059FD00F00DFA00F0FBF920F07B
S31508000478604020F07F00044B186000F0F3F94468E8
S31508000488FFF7A0FEA047E7E708ED00E070B508E02B
S31508000498461C4D1C0B78037000F090FD3046294623
S315080004A82246531E9CB2002AF2D170BD38B50546BD
S315080004B8002401E00134E4B2092C15D800F07EFDC9
S315080004C804EB44029300094AD358AB42F2D804EB2A
S315080004D844029100054A0A44526813449D42E9D2E7
S315080004E8024B0B44187A38BDFF2038BD80690008CE
S315080004F808B5C1F3080353B90368994209D040F807
S31508000508041B4FF40072FFF7C1FF012008BD002045
S3150800051808BD012008BD2DE9F04107460068FFF728
S31508000528C5FFFF282DD003F031FBF32003F046FB67
S3150800053803F04AFB012816D000247F2C17D83E68FA
S31508000548A30006EB03083B445D6800F037FD29461F
S31508000558404603F0A9FB08280BD156F824309D42DB
S315080005680DD10134E9E703F021FB002404E0012456
S3150800057800E0002403F01AFB2046BDE8F0810024B9
S31508000588F8E70024F8E7000038B50D460B4B984203
S3150800059808D004460A4B994206D0FFF7BCFF20B993
S315080005A8002407E0074C00E0044C29462046FFF7DC
S315080005B89FFF08B1204638BD0024FBE7D404002075
S315080005C800800008D00200202DE9F04106460C46B6
S315080005D817461D4621F4FF7828F001080368B3F189
S315080005E8FF3F0DD03368984505D041463046FFF79A
S315080005F8CBFF064628B33368E41A344404340CE0BF
S315080006084146FFF775FF03460028EBD116E017F8B1
S31508000618013B04F8013B013D0FD000F0CFFC331D28
S31508000628E31AB3F5007FF2D308F500713046FFF7F1
S31508000638ABFF064638B1041DE9E701231846BDE8AD
S31508000648F0810023FAE70023F8E7000088422CD84F
S3150800065838B504460D46012829D90B2901D90020A1
S3150800066838BD03F093FAF32003F0A8FA03F0ACFABE
S3150800067801280ED0AC4214D800F0A0FC02210D4B7C
S3150800068833F8140003F0D8FA082806D10134E4B27E
S31508000698F0E703F08BFA002038BD03F087FA00204C
S315080006A838BD03F083FA012038BD002070470020C2
S315080006B838BD00BFF86900084FF0FF33024A1360D7
S315080006C8024A1360704700BFD0020020D4040020F5
S315080006D870B504460D461646FFF7E8FEFF281AD0F9
S315080006E860190138FFF7E2FEFF2816D024F4FF73D5
S315080006F823F001030A4A934206D02B46324621467E
S315080007080848FFF761FF70BD2B4632462146064862
S31508000718FFF75AFF70BD002070BD002070BD00BFEE
S3150800072800800008D0020020D404002070B50446D2
S315080007380E46FFF7BBFE0546A0190138FFF7B6FEB9
S31508000748FF2D06D0FF2806D001462846FFF77EFF6C
S3150800075870BD002070BD002070BD0000104B1B68DE
S31508000768B3F1FF3F1AD000B583B00D4A53689168B4
S315080007780B44D1680B4411690B4451690B449169C0
S315080007880B44D26913445B4202AA42F8043D042189
S315080007980448FFF79DFF03B05DF804FB0120704786
S315080007A8D4040020888100080D4B1B680D4A12687E
S315080007B813440D4A126813440C4A126813440C4A27
S315080007C8126813440B4A126813440B4A12681344F6
S315080007D80A4A1268D34201D00020704701207047A0
S315080007E80080000804800008088000080C800008BB
S315080007F810800008148000081880000888810008FE
S3150800080808B50C4B1B68B3F1FF3F04D00948FFF73E
S3150800081882FE034650B1084B1B68B3F1FF3F07D069
S315080008280548FFF778FE034600B10123184608BDB8
S315080008380123FBE7D4040020D002002000487047B3
S315080008480080000808B5FFF737FF08BD08B5FFF7A9
S315080008583FFF08BD08B5FFF769FF08BD08B5FFF7EC
S31508000868A3FF08BD08B5FFF7E9FF08BD08B5FFF7F8
S3150800087875FF034608B9184608BDFFF7C1FF0346C2
S31508000888F9E700000022014B1A60704710E000E003
S3150800089808B5FFF7F7FF054B054A5A6000229A6024
S315080008A805211960034B1A6008BD00BF10E000E077
S315080008B83F900200D8060020044B1B6813F4803FBB
S315080008C803D0034A136801331360704710E000E049
S315080008D8D806002008B5FFF7EFFF014B186808BDD2
S315080008E8D806002010B504468021094803F0D2FB33
S315080008F808B9002010BD2146054803F0C3FB80212E
S31508000908034803F0C7FB0028F9D0012010BD00BF33
S315080009180044004010B504462021064803F0BAFBF7
S31508000928012801D0002010BD024803F0AFFB207053
S31508000938012010BD0044004010B584B04FF461434F
S3150800094800930023ADF80430ADF80630ADF808304A
S31508000958ADF80C300C23ADF80A30054C694620462C
S3150800096803F01AFB0121204603F07EFB04B010BDF4
S315080009780044004070B506460D4640290AD8284660
S31508000988FFF7B0FF012803D07A210E4800F032FAA3
S31508000998002406E076210B4800F02CFAEFE701342C
S315080009A8A4B2ABB29C420BD200F008FB305DFFF74D
S315080009B899FF0128F3D08321024800F01BFAEEE7D5
S315080009C870BD00BF286A000838B5224B1C78ACB938
S315080009D82148FFF79FFF012801D0204638BD1E4B46
S315080009E81B78002BF9D0FFF775FF1C4B18600022FF
S315080009F81B4B1A700122174B1A70EEE70546184B5F
S31508000A081B78013314481844FFF784FF0446012865
S31508000A180AD0FFF75FFF114B1B686433984216D953
S31508000A2800240C4B1C70D8E70D4B1A780132D2B249
S31508000A381A70094B1B789A4201D00024CDE7094958
S31508000A482846FFF723FD0022024B1A70C5E7002443
S31508000A58C3E700BF1D070020DC060020200700208A
S31508000A681E070020DD060020094B03F118010022A5
S31508000A7832B19A7400225A61054A064B1A607047C1
S31508000A889A745961183318310132D2B2F0E700BFA7
S31508000A98580D0020880D00200A4B1B6883B110B436
S31508000AA85C69084A146019749860D86000225A74F8
S31508000AB81860013908445860987C5DF8044B7047FB
S31508000AC8FF207047880D002038B504460D460128D2
S31508000AD804D94FF4CD71124800F08CF9620022440B
S31508000AE8D100104B0B445A7C1B7C9A4213D00D4BF1
S31508000AF80B44DA6815705A7C01325A74DA6801327E
S31508000B08DA605B689A4208D9064A08465158024488
S31508000B18D160012038BD002038BD012038BD00BF8E
S31508000B28546A0008580D002008B50146024B187883
S31508000B38FFF7CAFF08BD00BF8C0D002038B504466C
S31508000B480D46012804D94FF4DE71134800F052F90E
S31508000B5804EB4403DA00114B13445B7CBBB1620017
S31508000B682244D1000D4B0B449A6812782A705A7C95
S31508000B78013A5A749A6801329A605B689A4208D9A7
S31508000B88064A0846515802449160012038BD00209B
S31508000B9838BD012038BD00BF546A0008580D00202A
S31508000BA808B50146024B1878FFF7C8FF08BD00BF0D
S31508000BB8D00D002010B50446012804D94FF4EE716B
S31508000BC8044800F017F904EB4404E200024B134406
S31508000BD8587C10BD546A0008580D002030B583B0FB
S31508000BE8FFF742FF0F4C4021601CFFF755FF2070A6
S31508000BF80D4D4021681CFFF74FFF28702378FF2BFF
S31508000C080BD0FF2809D0094B0093094B094A012143
S31508000C18094804F051F803B030BD7921074800F0B7
S31508000C28E9F8F0E78C0D0020D00D0020C800002058
S31508000C3848000020AC00002024070020546A000859
S31508000C4808B5034805F0EBF8002002F0A3FE08BD36
S31508000C582407002070B506460D463F290AD82846B7
S31508000C68FFF762FF012803D09E210E4800F0C2F85C
S31508000C78002406E09A210B4800F0BCF8EFE7013497
S31508000C88A4B2ABB29C420BD200F098F9305DFFF7DC
S31508000C984BFF0128F3D0A721024800F0ABF8EEE78E
S31508000CA870BD00BF546A000838B505461B4805F0EC
S31508000CB85CFB1B4B1C788CB91A48FFF771FF012897
S31508000CC801D0204638BD174B1B78002BF9D00122D6
S31508000CD8134B1A700022144B1A70F2E7124B1B7842
S31508000CE8013310481844FFF75BFF0446012801D072
S31508000CF80024E6E70C4B1A780132D2B21A70094B6F
S31508000D081B789A4201D00024DBE708492846FFF7F2
S31508000D18BDFB0022024B1A70D3E700BF2407002048
S31508000D28540E0020140E0020550E0020150E002023
S31508000D3830B583B0144B1878FFF73CFF08B305465F
S31508000D48402800D94025002405E09DF807200F4BC8
S31508000D581A550134E4B2A5420DD90DF107010A4B1B
S31508000D681878FFF7EBFE0128EFD04FF49271084880
S31508000D7800F040F8E9E72B46044A8121054804F0C3
S31508000D88DEFF03B030BD00BF8C0D0020180D002013
S31508000D98546A00082407002070B500EB8000C200DA
S31508000DA8114B1344B3F88C63002401E00134A4B250
S31508000DB8B4420FD20D4B1D7805F0E6FC015D2846B6
S31508000DC8FFF782FE0128F1D040F24311084800F0E7
S31508000DD811F8EBE705F0D8FC402302460121024842
S31508000DE804F07FFF70BD00BF24070020D00D002047
S31508000DF8546A000808B500F0E1F8FCE708B500F001
S31508000E08D5F8012806D000F069F918B10B4B1B78FC
S31508000E18012B00D008BDFFF75DFD094B1B6803F5DC
S31508000E28FA639842F6D30022044B1A7000F060F968
S31508000E380028EFD1FFF70CFBECE700BF560E0020A1
S31508000E48580E002008B50122044B1A70FFF742FD18
S31508000E58034B1860FFF7D2FF08BD00BF560E0020E7
S31508000E68580E002008B5FFF7EFFA00F0A3F8FFF7C9
S31508000E780FFDFFF7E7FC00F019F900F00FF8FFF788
S31508000E88E1FF08BD08B500F099F8FFF715FD00F071
S31508000E983DFA00F017F8FFF7B1FF08BD10B502F0E4
S31508000EA8CDFCFFF7BDF9064C01232370FFF744FD77
S31508000EB800232370FFF792FE0223237010BD00BF9C
S31508000EC80000002008B51248FFF778FA01280AD06A
S31508000ED80F48FFF779FD01280CD00D48FFF7E4FE07
S31508000EE801280ED008BD01220A4B1A70084802F0DC
S31508000EF8C5FCEDE70022074B1A70054802F0BEFC50
S31508000F08EBE70222034B1A70014802F0B7FCE9E73F
S31508000F185C0E00200000002008B5FFF791FE08BD0A
S31508000F2838B504460D460E4B1B78012B09D00C4BD9
S31508000F381B7853B10A4B1B78022B0BD002F096FC90
S31508000F4838BDC9B2FFF7F0F9F1E7E9B22046FFF76D
S31508000F5811FDEFE7E9B22046FFF77CFEEEE700BF92
S31508000F6800000020074B1B78022B05D0032B05D061
S31508000F78012B05D0402070473F2070470020704756
S31508000F880820704700000020074B1B78022B05D065
S31508000F98032B05D0012B05D0402070473F2070470A
S31508000FA800207047082070470000002008B502F0A6
S31508000FB853FC08BD08B502F0E3FC08BD08B502F005
S31508000FC8E4FC08BD10B4034601310D4AA2FB03230D
S31508000FD8DB08F9D100230B70094BA3FB0023DB08B8
S31508000FE81A4603EB83035C00031B303301F8013D03
S31508000FF81046002AF0D108465DF8044B704700BF32
S31508001008CDCCCCCC00F00F03092802D903F1370060
S31508001018704710B503F1300405F046FC20444378C0
S3150800102803F00303022B01D0E0B210BD203CFBE716
S3150800103838B505460C460009FFF7E4FF207005F0A9
S315080010480F00FFF7DFFF60700023A370204638BD46
S31508001058F8B5074600252E4607E0203C10E0330180
S31508001068DBB21344DEB20135EDB2012D19D87C5D29
S3150800107805F01AFC2044437803F00303022BECD04E
S31508001088E3B2A3F13002D2B2162A09D8A3F13A017B
S31508001098C9B2062907D9092AE1D9373BDAB2DEE700
S315080010A800263046F8BD0026FBE7000008B50022F2
S315080010B8064B1A700649074801F052FD00B908BDE3
S315080010C877210548FFF796FEF9E700BFFC120020CE
S315080010D87C6A0008A40E0020806A0008034B1B7867
S315080010E80BB1002070470120704700BFFC12002092
S315080010F808B5FFF75BFF01280ED0084B1B780BB124
S31508001108002008BD02F07AFC012801D0002008BD9D
S315080011180122024B1A7008BD002008BDFC120020E7
S3150800112838B50546047805F0BFFB2044437803F034
S315080011380303022B03D0532C03D0032038BD203CCD
S31508001148F9E705F0B1FB6B781844427812F0040FFA
S3150800115801D1032038BD312B07D0322B07D0332BCA
S3150800116801D0032038BD022038BD002038BD012033
S3150800117838BD70B506460230FFF76AFF054684B2E1
S3150800118804363046FFF764FF0544EDB2013CA4B2C5
S315080011980236012CF5D8ED43EDB23046FFF758FF75
S315080011A8854201D0002070BD012070BD2DE9F041AF
S315080011B8044616468846A1B198B12046FFF7B0FFFF
S315080011C80546032800F099802046FFF7D2FF002835
S315080011D800F09780012D2DD04DB1022D57D000274C
S315080011E88CE040F261214848FFF704FEE5E7A01CB9
S315080011F8FFF72EFF87B2201DFFF72AFF0002C8F85F
S315080012080000A01DFFF724FFD8F800301844C8F8D6
S3150800121800000834033F3FB2002E6FD0002506E0D1
S315080012282046FFF715FF705502340135ADB2BD42A9
S31508001238F6DB63E0A01CFFF70BFF87B2201DFFF75C
S3150800124807FF0004C8F80000A01DFFF701FFD8F83B
S31508001258003003EB0020C8F8000004F10800FFF787
S31508001268F7FED8F800301844C8F800000A34043FD6
S315080012783FB2002E42D0002506E02046FFF7E8FEDA
S31508001288705502340135ADB2BD42F6DB36E0A01C16
S31508001298FFF7DEFE87B2201DFFF7DAFE0006C8F85C
S315080012A80000A01DFFF7D4FED8F8003003EB004075
S315080012B8C8F8000004F10800FFF7CAFED8F800309D
S315080012C803EB0020C8F8000004F10A00FFF7C0FE87
S315080012D8D8F800301844C8F800000C34053F3FB267
S315080012E866B1002506E02046FFF7B2FE70550234BF
S315080012F80135ADB2BD42F6DB00E000273846BDE849
S31508001308F0814FF0FF37F9E7806A0008964B1B789B
S31508001318002B00F0F18170B5012B05D0022B2DD0DA
S31508001328032B00F03F8170BDFFF78CFA02F088FBAB
S315080013388E4802F0C9FB8E4802F0C6FB02F07CFB19
S31508001348012201468B4801F037FC30B18A4802F081
S31508001358BBFB012002F0AAFB70BD884802F0B4FB6B
S31508001368874802F0B1FB874802F0AEFB864B00229D
S315080013781A605A6002227C4B1A7070BD834C04F5B9
S315080013880C724FF48071824802F030F894F84132B2
S31508001398002B5ED1002877D07D48002200F5C07161
S315080013A8FFF704FF0446B0F1FF3F60D0002C09DDC3
S315080013B8754B5B68002B69D1754BD3F88021724B46
S315080013C81A605C60714BD3F84422D3F83C329A42CF
S315080013D8A9D10021674801F0C5FE002840F0A98078
S315080013E8694B5B6873B3654802F06EFB694802F09F
S315080013F86BFB694D644C29466068FFF7E3FD284690
S3150800140802F062FB654802F05FFB2946E078FFF7C1
S315080014180FFEA91CA078FFF70BFE291D6078FFF7B9
S3150800142807FEA91D2078FFF703FE284602F04CFBA5
S315080014385B4802F049FB61682068FFF70BFA002849
S3150800144800F084804D4802F03FFB0322464B1A7091
S3150800145870BD494802F038FB022002F027FB04F564
S315080014680C7001F06BFE00223F4B1A7070BD4248A3
S3150800147802F02AFB032002F019FB3E4801F05EFE43
S315080014880022394B1A7070BD00248FE7404AD2F8FB
S3150800149880113D4A12681A44914239D0374802F0F9
S315080014A813FB3C4802F010FB3B4E374D3146686843
S315080014B8FFF788FD304602F007FB384802F004FBC0
S315080014C83146E878FFF7B4FDB11CA878FFF7B0FDF8
S315080014D8311D6878FFF7ACFDB11D2878FFF7A8FD20
S315080014E8304602F0F1FA2E4802F0EEFA69682868E2
S315080014F8FFF7B0F980B1214802F0E6FA214802F070
S31508001508E3FA234BD3F880211F4B1A605C6059E72E
S3150800151823441D4A536055E7174802F0D5FA0520B3
S3150800152802F0C4FA134801F009FE00220E4B1A709D
S3150800153870BD114802F0C8FA042002F0B7FA0D483F
S3150800154801F0FCFD0022084B1A7070BD0A4802F02B
S31508001558BBFA052002F0AAFA064801F0EFFD0022B8
S31508001568014B1A7070BD00BFFC1200209C6A000867
S31508001578C06A0008D4100020E86A0008F06A000863
S31508001588F86A00081C6B00089C0E0020A40E0020B0
S31508001598001300204C6B000884140020586B0008C0
S315080015A8FC6B0008554C04F50C724FF480715448CE
S315080015B801F01CFF94F84132002B66D100287FD031
S315080015C84F4800F5807200F5C071FFF7EFFD054634
S315080015D8B0F1FF3F67D0002D34DD4A4802F074FAAF
S315080015E8494C21462846FFF7EDFC204602F06CFADE
S315080015F8464802F069FA424E214696F88301FFF7F3
S3150800160817FDA11C96F88201FFF712FD211D96F811
S315080016188101FFF70DFDA11D96F88001FFF708FD6A
S31508001628204602F051FA3A4802F04EFA06F5807258
S315080016382946D6F88001FFF709F9002842D0354827
S3150800164802F042FA2D4BD3F84422D3F83C329A4298
S315080016587FF469AE304802F037FAFFF707F9002831
S315080016683DD02C4802F030FA2C4802F02DFA2C48C6
S3150800167801F064FD2B4802F027FA00222A4B1A705B
S3150800168802F0F2F9FEF7E4FE4DE6284802F01CFAE5
S31508001698022002F00BFA04F50C7001F04FFD002247
S315080016A8214B1A7070BD224802F00EFA032002F088
S315080016B8FDF91B4801F042FD00221B4B1A7070BD4C
S315080016C8002588E71B4802F0FFF9062002F0EEF924
S315080016D8134801F033FD0022134B1A7070BD1548E4
S315080016E802F0F2F9072002F0E1F90D4801F026FDAB
S315080016F800220D4B1A7070BD704700BFA40E00205B
S3150800170800130020BC6B000884140020CC6B00086A
S31508001718FC6B0008F06A0008E46B0008006C000817
S31508001728D4100020186C0008FC120020746B0008FE
S31508001738986B0008E86A00084278007840EA0220B0
S315080017487047C278837843EA0222437843EA022339
S31508001758007840EA032070470170090A417070470B
S315080017680170C1F307234370C1F307438370090E59
S31508001778C170704713462AB10A78027001300131E0
S31508001788013BF9D1704701700130013AFBD1704726
S3150800179830B4451C037808781B1A013A04D04C1C47
S315080017A828462146002BF4D0184630BC704700E07E
S315080017B8013003780BB18B42FAD1184670470239C3
S315080017C84369023B994204D24389806A03FB0100B4
S315080017D870470020704770B506460D4601F11A0095
S315080017E8FFF7AAFF04463378032B00D070BD05F12E
S315080017F81400FFF7A1FF44EA0040F7E770B506466C
S315080018080C46154691B204F11A00FFF7A5FF33787E
S31508001818032B00D070BD290C04F11400FFF79CFFB8
S31508001828F8E700002DE9F04180460F4601F11A0055
S31508001838FFF782FF58BB3D7805F03F05013D05EBEC
S31508001848450305EB83050126002404E04FF6FF73DC
S31508001858984222D101340C2C0DD8144B185D384403
S31508001868FFF76AFF002EF1D0FE2D13D828F81500C9
S3150800187806460135EEE73B7813F0400F10D0FE2DEB
S3150800188811D8002328F815300120BDE8F08100207A
S31508001898BDE8F0810020BDE8F0810020BDE8F081B0
S315080018A80120BDE8F0810020BDE8F081C46C00087D
S315080018B82DE9F84380460F4691464B730F23CB72A2
S315080018C800240C73214607F11A00FFF745FF09F1B2
S315080018D8FF3606EB460306EB8306254602E0013487
S315080018E80C2C11D84FF6FF739D4202D038F81650C3
S315080018F801360C4B185D29463844FFF72DFF002D95
S31508001908EDD14FF6FF75EAE74FF6FF739D4202D011
S3150800191838F816300BB949F0400987F80090BDE841
S31508001928F88300BFC46C000870B582B00546164631
S315080019381C460B22FFF71EFF052C11D807231FE0AC
S3150800194801310F290DD802F0010000EB43035208B4
S3150800195813F4803FF4D083F4883383F02103EFE748
S315080019682346328812B102360021EAE71C46E5E723
S315080019785A1E02A8034403F8081C240909D013466A
S3150800198804F00F0202F130013929F1D902F13701C1
S31508001998EEE77E210346134403F8081C00E00134E9
S315080019A8944208D22B5D202BF9D104E02020187028
S315080019B80C46072909D8611C2B19072AF6D802A844
S315080019C8104410F8080C0132F1E702B070BD014660
S315080019D80B220020C30143EA5003087850FA83F320
S315080019E8D8B20131013AF5D17047016809B10A46FA
S315080019F803E04FF0FF3308E0013213781F2B01D9B3
S31508001A083A2BF9D13A2B02D000231846704710B45E
S31508001A184C1C0B78303B092B08D8A24209D15BB974
S31508001A280132026018465DF8044B70474FF0FF33E1
S31508001A38F8E74FF0FF33F5E74FF0FF33F2E738B52D
S31508001A480C4620B1054603680BB11A781AB9002363
S31508001A582360092038BDD98882889142F7D15878F9
S31508001A6802F0A0FD10F0010FF1D12B6823600020C9
S31508001A7838BDF8B5C3780BB90020F8BD0446C66A60
S31508001A8800F13007012332463946407802F0D8FD7E
S31508001A98A8B90023E370236AF31AA269934210D2FD
S31508001AA8A57808E0A3691E440123324639466078BA
S31508001AB802F0C6FD013D012DF4D80020F8BD01202D
S31508001AC8F8BD0020F8BD70B5C36A8B4214D0044629
S31508001AD80D46FFF7CEFF064608B1304670BD01230E
S31508001AE82A4604F13001607802F066FD10B1012635
S31508001AF84FF0FF35E562F0E70026EEE710B5044635
S31508001B080023C3704FF0FF33C362FFF7DCFF08B149
S31508001B18042010BD04F22E20FFF70EFE4AF65523C0
S31508001B28984201D0032010BD04F16600FFF709FEAC
S31508001B3820F07F40084B98420CD004F18200FFF74A
S31508001B4800FE20F07F40044B984201D0022010BDC9
S31508001B58002010BD002010BD464154002DE9F0476D
S31508001B6884B00E46174600230B60FFF73EFF051E96
S31508001B78C0F23581A84B53F82540002C00F0338174
S31508001B88346007F0FE0723787BB1607802F00AFD17
S31508001B9810F0010F09D1002F00F0278110F0040F6B
S31508001BA801D00A201CE100201AE100232370E8B2BC
S31508001BB8607002F051FC10F0010F01D003200FE10C
S31508001BC827B110F0040F01D00A2009E100212046A8
S31508001BD8FFF794FF02281DD00026042800F0078185
S31508001BE801282DD90D20FBE0002004AB03EB850363
S31508001BF843F8100C0135032D0ED804F130002B01DB
S31508001C0803F5DF7318440379002BEDD00830FFF786
S31508001C1898FDEAE70025EEE7002508E03146204664
S31508001C28FFF76CFF0128D8D90135032DD5D804ABA1
S31508001C3803EB850353F8106C002EEFD10320F1E768
S31508001C4804F13B00FFF778FDB0F5007F01D00D20C1
S31508001C58C6E004F14600FFF76FFD804620B904F197
S31508001C685400FFF76EFD8046C4F8188094F8409033
S31508001C7884F8029009F1FF33DBB2012B01D90D2054
S31508001C88AEE009FB08F994F83D706781002F00F06B
S31508001C98B0807B1E1F4201D00D20A1E004F141004F
S31508001CA8FFF74AFD8246208110F00F0F40F0A38007
S31508001CB804F14300FFF740FD054620B904F150003A
S31508001CC8FFF73FFD054604F13E00FFF735FD0246DE
S31508001CD8002800F0928009EB000303EB1A139D42D3
S31508001CE8C0F08D80ED1AB5FBF7F5002D00F0898058
S31508001CF840F6F5718D4260D801274FF6F5718D4289
S31508001D0800D9032702356561E66132442262334405
S31508001D18A362032F53D104F15A00FFF70DFD0028DB
S31508001D2871D1BAF1000F70D104F15C00FFF709FD13
S31508001D386062AD0005F2FF15B8EB552F69D34FF071
S31508001D48FF332361E36080232371032F2CD104F129
S31508001D586000FFF7F1FC012826D1711C2046FFF721
S31508001D68B2FE08BB0023237104F22E20FFF7E4FC19
S31508001D784AF65523984217D104F13000FFF7E1FCDB
S31508001D88264B984210D104F50570FFF7DAFC244B68
S31508001D98984209D104F50670FFF7D3FC206104F5CB
S31508001DA80770FFF7CEFCE06027701E4A13880133D8
S31508001DB89BB21380E380002012E002279DE7BAF160
S31508001DC8000F24D04A446262022F01D16D00B1E7A0
S31508001DD805EB450305F0010505EB5305AAE70B20B6
S31508001DE804B0BDE8F0870C20FAE70020F8E70120E0
S31508001DF8F6E70D20F4E70D20F2E70D20F0E70D20B1
S31508001E08EEE70D20ECE70D20EAE70D20E8E70D20C0
S31508001E18E6E70D20E4E700BFC414002052526141EA
S31508001E2872724161C8140020F8B5066801295DD99F
S31508001E38736999425CD20C463378022B30D0032B4F
S31508001E4840D0012B01D00120F8BD01EB5105316ABC
S31508001E5801EB55213046FFF736FE10B14FF0FF303B
S31508001E68F8BD6F1CC5F30805354495F83050316A36
S31508001E7801EB57213046FFF726FE10B14FF0FF3029
S31508001E88F8BDC7F308073E4496F8300045EA00202F
S31508001E9814F0010F01D00009F8BDC0F30B00F8BD16
S31508001EA8316A01EB14213046FFF70DFE10B14FF0E9
S31508001EB8FF30F8BD600000F4FF7030303044FFF79B
S31508001EC83BFCF8BD316A01EBD4113046FFF7FBFD40
S31508001ED810B14FF0FF30F8BDA00000F4FE703030A6
S31508001EE83044FFF72EFC20F07040F8BD0120F8BDFD
S31508001EF80120F8BD2DE9F0410768B1F5001F02D3A6
S31508001F080220BDE8F08106460C4611F01F0F02D0E4
S31508001F180220BDE8F081316185681DB93B78022B3E
S31508001F2800D97D6A75B93B89B3EB541F02D80220DC
S31508001F38BDE8F0817B6AB3617561B3690BBB0220A2
S31508001F48BDE8F081B7F80A804FEA482801E0A4EB13
S31508001F58080444450FD329463046FFF765FF05466A
S31508001F68B0F1FF3F18D0012819D97B699842EED3FA
S31508001F780220BDE8F08129463846FFF720FCB06103
S31508001F88DAE703EB5423B3613037C4F308043C4457
S31508001F98F4610020BDE8F0810120BDE8F081022047
S31508001FA8BDE8F0812DE9F84301297ED943699942AC
S31508001FB801D302267AE017460C4605460378022B13
S31508001FC847D0032B57D0012B01D002266EE001EB30
S31508001FD85108016A01EB5821FFF775FD06460028E6
S31508001FE864D108F10109C8F3080814F0010423D0DC
S31508001FF805EB080393F9303003F00F033A0102F4AE
S315080020087F621343DBB2A84488F830300123EB70AB
S31508002018296A01EB59212846FFF755FD0646002887
S3150800202844D1C9F308094CB1C7F30712A94489F87A
S3150800203830200123EB7039E0FBB2E4E705EB09032E
S3150800204893F9302022F00F02C7F303273A43D2B296
S31508002058ECE7016A01EB1421FFF735FD064628BBB4
S31508002068600000F4FF703030B9B22844FFF774FBFB
S315080020780123EB701AE0016A01EBD411FFF723FD7F
S31508002088064698B927F07047A40004F4FE7430345D
S315080020982C442046FFF755FB00F07041394320468B
S315080020A8FFF75EFB0123EB7000E002263046BDE829
S315080020B8F8832DE9F04107460668884631B9F56878
S315080020C88DB173699D420FD301250DE0FFF7ACFE6C
S315080020D80346012847D9B0F1FF3F49D072699042B3
S315080020E846D3454600E001252C460CE021463846ED
S315080020F8FFF79AFE034670B1012839D0B0F1FF3FC1
S3150800210836D0AC4233D0013473699C42EED3012DE4
S315080021182BD90224EAE74FF0FF3221463046FFF76B
S3150800212841FF034610B9B8F1000F0ED1A3B9F46000
S3150800213833697269023A934201D2013B33613379B2
S3150800214843F001033371234612E0224641463046DE
S31508002158FFF728FF0346E9E7012B01D0012307E02B
S315080021684FF0FF3304E0012302E0002300E00023D8
S315080021781846BDE8F081F8B50E460468012930D935
S315080021880746114663699E4201D302222AE05AB1DC
S315080021984FF0FF322046FFF705FF024620B121E03F
S315080021A863692E469D421DD231463846FFF73CFEE6
S315080021B80546C8B1012819D0B0F1FF3F18D000224A
S315080021C831462046FFF7EEFE024658B92369B3F1B1
S315080021D8FF3FE5D001332361237943F001032371D7
S315080021E8DEE702221046F8BD0022FBE70222F9E7DD
S315080021F80122F7E72DE9F8430668036903F1200584
S31508002208836913B90420BDE8F883B5F5001F02D31E
S315080022180420BDE8F88388460446C5F308078FB93D
S3150800222801338361416941B93389B3EB551F09D82D
S31508002238002383610420BDE8F8837389013B13EA08
S31508002248552307D0256107F130084644E661002082
S31508002258BDE8F883FFF7E8FD8146012848D9B0F1BB
S31508002268FF3F48D0736998423AD3B8F1000F04D1B2
S315080022780023A3610420BDE8F88361692046FFF7B7
S3150800228818FF814610B90720BDE8F883012835D01C
S31508002298B0F1FF3F35D03046FFF7EBFBA0BB4FF454
S315080022A80072002106F13000FFF76DFA49463046FC
S315080022B8FFF785FAF0624FF00008738998450BD244
S315080022C80123F3703046FFF7D4FB00BB08F1010879
S315080022D8F36A0133F362F0E7F36AA3EB0803F362E0
S315080022E8C4F8149049463046FFF769FAA061A9E789
S315080022F80220BDE8F8830120BDE8F8830220BDE87E
S31508002308F8830120BDE8F8830120BDE8F883012099
S31508002318BDE8F883F8B504460F4606680021FFF7B6
S31508002328E9FD0246C0B9002508E00135BD4213D0CB
S3150800233801212046FFF75EFF024668B9A1693046C3
S31508002348FFF7C1FB024638B9E3691B78E52BECD0E1
S31508002358002BEAD00025EBE7042A01D01046F8BD81
S315080023680722FBE72DE9F8430446884607684FF035
S31508002378FF094E4604252EE00F2B19D112F0400FFF
S3150800238806D091F80D9002F0BF02236963621646DB
S31508002398B24201D0FF2618E04B7B994501D0FF26AB
S315080023A813E0A06AFFF73EFA88B3013EF6B20CE0DE
S315080023B826B90846FFF70BFB81452BD04FF0FF33AC
S315080023C8636227E0FF2600E0FF2600212046FFF784
S315080023D811FF0546F0B9A169E1B13846FFF773FB65
S315080023E80546B8B9E1690A789AB1CB7A03F03F038A
S315080023F8A371E52AE6D02E2AE6D023F0200008287D
S3150800240814BF002001204045B6D0FF26DDE7FF2689
S31508002418DBE704250DB10023A3612846BDE8F88348
S3150800242870B5044605680669416AB1F1FF3F1CD0D4
S31508002438FFF760FD0346B3B9A1692846FFF743FBD2
S31508002448034670B9E269E52111700122EA7022692A
S31508002458964206D900212046FFF7CCFE03460028F7
S31508002468EAD0042B03D0184670BD0023E3E70223FD
S31508002478F9E700002DE9F04F83B006468A46D1F8F9
S315080024880090856A002412E0013709EB070219F85B
S3150800249807302F2BF8D05C2BF6D0CAF800201F2857
S315080024A822D84FF0040823E025F814803C46671C18
S315080024B819F804001F28E8D92F28E6D05C28E4D0A4
S315080024C8FE2C00F2DD80012100F0E2FF804600289C
S315080024D800F0D8807F28E7D801466B48FFF767F9E8
S315080024E80028E1D0062012E04FF0000800E0013C81
S315080024F844B104F10043013B35F81330202BF6D0DC
S315080025082E2BF4D0002325F814301CB9062003B066
S31508002518BDE8F08F0B222021306AFFF734F9002333
S3150800252800E0013335F81320202AFAD02E2AF8D0ED
S315080025381BB148F0030800E0013C6CB104F1004205
S31508002548013A35F812202E2AF6D14FF0080B4FF02B
S31508002558000ACDF804A00AE0A2464FF0080B0022AC
S31508002568019204E04C450BD048F003084B4603F1AA
S31508002578010935F8137057B3202FF5D02E2FF1D04F
S31508002588DA450FD24C450DD07F2F3FD8002F4AD1B8
S3150800259848F003085F27336A03F80A704B460AF1BE
S315080025A8010AE4E7BBF10B0F0FD04C4501D048F000
S315080025B803084C450BD3019B9B00DBB201932346CA
S315080025C84FF00B0B4FF0080AD1E748F00308336AB7
S315080025D81A78E52A43D0BBF1080F43D0019901F0D0
S315080025E80C020C2A43D001F00303032B3FD018F042
S315080025F8020F06D1019B03F00303012B3AD0042AE4
S315080026083BD0336A83F80B80002080E700213846E0
S3150800261800F03EFF074618B1A0F180071B4BDF5DA7
S3150800262848F00208B2E739461948FFF7C0F8002803
S31508002638AED1A7F141039BB2192B04D8019B43F0ED
S3150800264802030193A7E7A7F161039BB2192BA2D846
S31508002658019B43F001030193203FBFB29BE7052284
S315080026681A70B8E7019B9B00DBB20193B6E748F0FE
S315080026780208BCE748F01008C1E748F00808C0E7B0
S31508002688062044E7062042E7D46C0008446C000894
S31508002698E06C0008F8B500238B758369002B6BD0AE
S315080026A80D460646436AB3F1FF3F13D0836A0024F2
S315080026B89F1C188858B1002100F0EAFE30B1FE2C9C
S315080026C80CD82A1990753B460134F1E700242C44A6
S315080026D80023A375AC7D0022134612E00024F6E712
S315080026E8E52317E014B9A8182E278775A8182E27E2
S315080026F84772013210E010271CE0A81883750132CA
S315080027080B460A2B1BD8F069591CC35C202BF7D03B
S31508002718052BE5D00929E5D0A8184372002CEED177
S31508002728A3F14100C0B21928E7D8F069007B082947
S31508002738E1D808270742E0D02033DBB2DDE734B911
S31508002748AB1800219975F3691B7B03B90A462A4415
S3150800275800235372F369DB7A2B72F0691C30FEF793
S31508002768F0FF2860F0691830FEF7E6FFA880F069E0
S315080027781630FEF7E1FFE880F8BD00002DE9F047BE
S315080027888146884601F11A00FEF7D6FFB0BB98F8CD
S31508002798005005F03F05013D05EB450305EB8305AC
S315080027A80127002404E04FF6FF7398422FD101341D
S315080027B80C2C17D81C4B185D4044FEF7BDFF06467F
S315080027C8002FF0D0FE2D1CD800F07EFE074605F136
S315080027D8010A39F8150000F077FE874214D1374602
S315080027E85546E4E798F8003013F0400F12D0A7B121
S315080027F839F81530A3B90120BDE8F0870020BDE8EF
S31508002808F0870020BDE8F0870020BDE8F0870020A3
S31508002818BDE8F0870120BDE8F0870120BDE8F0870C
S315080028280020BDE8F08700BFC46C00082DE9F8430E
S315080028380446D0F800800021FFF75CFB064600280E
S315080028485ED14FF0FF3363624FF0FF094F460AE047
S315080028584FF0FF336362FF2700212046FFF7CAFCC3
S31508002868064600284CD1A1694046FFF72CF90646CA
S31508002878002845D1E5692B78002B40D0E97A01F084
S315080028883F02A271E52BE3D011F0080F01D00F2AF9
S31508002898DED10F2A14D027B92846FFF798F88145BC
S315080028A82ED0216ACB7A13F0010F04D10B222846C1
S315080028B8FEF76EFF20B34FF0FF336362FF27CBE7BF
S315080028C8A06A0028C8D013F0400F06D095F80D90D6
S315080028D803F0BF03226962621F46BB4201D0FF2785
S315080028E8BAE76B7B994501D0FF27B5E72946FFF775
S315080028F845FF10B1013FFFB2AEE7FF27ACE7042654
S315080029083046BDE8F88330B583B0044601910568BA
S3150800291801E001330193019B1A782F2AF9D05C2A22
S31508002928F7D00022A2601B781F2B1DD901A92046C3
S31508002938FFF7A0FD0346F8B92046FFF777FF236A95
S31508002948DA7A0346D8B912F0040F15D1A37913F029
S31508002958100F1BD02169C1F30801303129442846D4
S31508002968FEF739FFA060E1E7236A8022DA720021C0
S315080029782046FFF7BFFA0346184603B030BD0428B9
S31508002988FAD112F0040FF7D10523F5E70523F3E783
S315080029982DE9F04784B00668D0F820A0D0F828803A
S315080029A89AF80B3013F0A00F05D04FF006094846E1
S315080029B804B0BDE8F087002400E0013438F8143084
S315080029C8002BFAD105460C22514601A8FEF7D2FE7D
S315080029D89DF80F3013F0010F1ED000238AF80B302C
S315080029E8AB620127632F0CD83B46424601A95046DD
S315080029F8FEF79AFF2846FFF719FF814608B90137F7
S31508002A08F0E7642F60D0B9F1040FD0D19DF80F30E4
S31508002A188AF80B30C5F828809DF80F3013F0020F96
S31508002A282AD00C342A4BA3FB0434A40801342146C3
S31508002A382846FFF76FFC814608B9013C1ED1B9F153
S31508002A48000FB4D1A9693046FFF73DF8814600283A
S31508002A58ADD120220021E869FEF795FE0B22296AE6
S31508002A68E869FEF787FEEA692B6ADB7A03F018033A
S31508002A7813730123F3709AE70124D8E72969A1EBB0
S31508002A8844112846FFF736FA81460028D7D1286A1E
S31508002A98FEF79DFF0746A9693046FFF714F88146F1
S31508002AA80028CCD13B46E2B2E969A86AFEF700FFDE
S31508002AB80123F37000212846FFF79CFB814600286E
S31508002AC8BDD1013CE7D1BAE74FF007096FE700BF68
S31508002AD84FECC44E70B50446FEF7CBFF054648B919
S31508002AE82378032B08D000221146607801F0FEFDF2
S31508002AF800B10125284670BD2379012BF3D104F1CD
S31508002B0830064FF4007200213046FEF73CFE4AF6BE
S31508002B18552104F22E20FEF71FFE0F493046FEF710
S31508002B281FFE0E4904F50570FEF71AFE216904F51D
S31508002B380670FEF715FEE16804F50770FEF710FE45
S31508002B48E2690132E26201233146607801F078FDD4
S31508002B5800232371C7E700BF52526141727241616F
S31508002B6810B584B001900091144604A840F8041DD5
S31508002B78FEF73BFF002818DB0E4B53F820300BB145
S31508002B8800221A70019B0BB100221A70019B094A90
S31508002B9842F8203063B1012C01D0002006E000225B
S31508002BA801A96846FEF7DAFF00E00B2004B010BD5D
S31508002BB80020FBE7C41400202DE9F04393B00191E7
S31508002BC8002800F0AE80044616460023036002F08B
S31508002BD81F073A4606A901A8FEF7C0FF05460028BA
S31508002BE840F0A080069B079303AB0F934F4B1193B6
S31508002BF8019907A8FFF787FE054620B90F9B93F9A1
S31508002C080B30002B2FDB16F01C0F79D0002D31D096
S31508002C18042D2AD047F0080715B917F0080F35D13B
S31508002C284DB917F0080F01D047F02007069BDB6A55
S31508002C3823620E9B6362002D74D1069EDDF83880E8
S31508002C4841463046FEF7C7FDA06008F11C00FEF7AE
S31508002C5878FDE060002363746361E3612774266086
S31508002C68F388A3805EE00625CDE707A8FFF790FE60
S31508002C780546CFE79DF8223013F0110F04D116F058
S31508002C88040FC9D00825C7E70725C5E7284E3146E2
S31508002C980E980E30FEF764FD31460E981630FEF78C
S31508002CA85FFD20220E9BDA72069EDDF838804146C3
S31508002CB83046FEF790FD8146002241463046FEF72B
S31508002CC89DFD00210E981C30FEF74AFD0122069B41
S31508002CD8DA70B9F1000FA3D0069BDE6A00224946CE
S31508002CE807A8FFF748FA0546002899D131460698F5
S31508002CF8FEF7E9FE054609F1FF33069AD3608FE722
S31508002D08002D8DD19DF8223013F0100F07D116F03B
S31508002D18020F85D013F0010F82D0072580E7042516
S31508002D287EE70925284613B0BDE8F083CC140020B1
S31508002D38000061482DE9F04F85B0044688461646D6
S31508002D4899460023C9F8003003A9FEF778FE074616
S31508002D5830B9677C27B9237C13F0010F04D10727FC
S31508002D68384605B0BDE8F08FE36862699B1AB34236
S31508002D7853D21E4651E0A1692046FFF755F85EE092
S31508002D8802276774ECE701276774E9E7022767747F
S31508002D98E6E701276774E3E74FF4007204F12801B0
S31508002DA808EB4020FEF7E6FC74E0E269019B9342D3
S31508002DB819D0237C13F0400F0BD0012304F1280106
S31508002DC8687801F03DFC002867D1237C23F040038E
S31508002DD823740123019A04F128010398407801F025
S31508002DE8EBFB00285CD1019BE3616169C1F308012B
S31508002DF8C1F50075AE4200D2354628312A46214427
S31508002E084046FEF7B7FCA84463692B446361D9F8C2
S31508002E1800302B44C9F80030761B002EA0D0636911
S31508002E28C3F30802002AE0D1039AB2F80AA00AF105
S31508002E38FF3A1AEA532A08D1002B9CD1A068012820
S31508002E489ED9B0F1FF3F9ED0A061039DA16928468F
S31508002E58FEF7B5FC002899D00AEB000301935FEA50
S31508002E68562BA2D00AEB0B036A89934201D9A2EB27
S31508002E780A0B5B46019A4146687801F09DFB0028D3
S31508002E8887D1237C13F0400F04D0E069019BC01A50
S31508002E98834581D84FEA4B25B5E7012767745FE76D
S31508002EA8012767745CE72DE9F04F85B00446884624
S31508002EB8164699460023C9F8003003A9FEF7BFFD50
S31508002EC8074630B9677C27B9237C13F0020F04D16B
S31508002ED80727384605B0BDE8F08F6369F3425FD324
S31508002EE8DE435DE000212046FFF7E3F86CE0A169C0
S31508002EF82046FFF7DEF867E002276774E9E7012747
S31508002F086774E6E70123E26904F128010398407823
S31508002F1801F096FB20B9237C23F04003237462E072
S31508002F2801276774D5E702276774D2E7012767740C
S31508002F38CFE74FF4007208EB412104F12800FEF7A9
S31508002F4819FC237C23F0400323746EE0E3699B4550
S31508002F5803D06269E3689A4269D3C4F81CB0606909
S31508002F68C0F30800C0F50075AE4200D235462830D1
S31508002F782A4641462044FEF7FDFB237C43F04003DE
S31508002F882374A84463692B446361E268934238BF93
S31508002F981346E360D9F800302B44C9F80030761B8D
S31508002FA8002E51D06369C3F30802002AD7D1039AC1
S31508002FB8B2F80AA00AF1FF3A1AEA532A0FD1002BE7
S31508002FC895D1A06800288DD000283DD0012893D037
S31508002FD8B0F1FF3F93D0A061A36803B9A060237C32
S31508002FE813F0400F8ED1039B0193A1691846FEF78B
S31508002FF8E6FB8346002896D0D344750AA6D00AEB82
S315080030080503019A5289934201D9A2EB0A052B4670
S315080030185A4641460198407801F012FB002885D1A6
S31508003028E169A1EB0B018D4283D86D02A9E701235B
S315080030385A4604F128010198407801F0BDFA00289B
S315080030488BD00127677444E7237C43F02003237455
S315080030583FE770B582B004460E460A290DD0636864
S31508003068002B08DB5D1C23441E733C2D09DC6560B8
S31508003078A3680133A36002B070BD0D21FFF7E9FF0D
S31508003088EDE701AB2A4604F10C012068FFF70BFFB0
S31508003098019B9D4202D04FF0FF35E8E70025E6E799
S315080030A830B583B0044601A9FEF7C9FC0346C8B97A
S315080030B8227C12F0200F15D012F0400F0CD00123F5
S315080030C8E26904F128010198407801F0B9FA88BB49
S315080030D8237C23F040032374216A0198FEF7F3FC46
S315080030E8034610B1184603B030BD656AEB7A43F05B
S315080030F82003EB72A26829462068FEF77FFBE16881
S3150800310805F11C00FEF72CFB0B4905F11600FEF726
S3150800311827FB002105F11200FEF71EFB0122019B81
S31508003128DA700198FFF7D6FC0346227C22F02002C3
S315080031382274D7E70123D5E70000614810B582B0A5
S315080031480446FFF7ADFF034610B1184602B010BD96
S3150800315801A92046FEF773FC03460028F5D100228C
S315080031682260F2E72DE9F04182B004460E4601A92D
S31508003178FEF765FC0746002840F0A280677C002F0A
S3150800318840F09E80E368B34204D2227C12F0020F14
S3150800319800D11E46636900226261002E65D0019A35
S315080031A8B2F80A804FEA482873B1721EB2FBF8F2E1
S315080031B8013BB3FBF8F18A4206D3C8F10002134073
S315080031C86361F61AA56902E0A56815B1A56135BB5C
S315080031D84CE000212046FEF76CFF0546012804D07E
S315080031E8B0F1FF3F04D0A060F0E70227677467E0F4
S315080031F80127677464E029462046FEF715FE05464A
S31508003208B5F1FF3F28D0012D29D9019B5B699D425D
S3150800321825D2A561636943446361A6EB080646455A
S315080032280BD9237C13F0020FE5D029462046FEF772
S3150800323840FF05460028E3D146466369334463617F
S31508003248C6F30803002B3FD029460198FEF7B7FABC
S3150800325840B90227677433E00127677430E002270C
S3150800326867742DE000EB562500E000256369C3F373
S315080032780803E3B1E269954219D0237C13F0400F9D
S315080032880BD0012304F128010198407801F0D8F9F8
S31508003298E0B9237C23F04003237401232A4604F16A
S315080032A828010198407801F087F990B9E5616369C2
S315080032B8E268934204D9E360237C43F0200323742D
S315080032C8384602B0BDE8F0810025CFE701276774C4
S315080032D8F6E701276774F3E730B591B001900D4614
S315080032E8002205A901A8FEF739FC044610B12046B4
S315080032F811B030BD02AB0D930B4B0F93019905A87E
S31508003308FFF701FB04460028F1D10D9B93F90B3012
S31508003318002B06DB002DEAD0294605A8FFF7BAF9DF
S31508003328E5E70624E3E700BFCC14002070B59CB097
S315080033380190022205A901A8FEF710FC059B119326
S31508003348044610B120461CB070BD02AB1993264B33
S315080033581B93019911A8FFF7D6FA04460028F1D15C
S31508003368199B93F90B30002B23DB9DF84A3013F091
S31508003378010F20D10CBB059E18993046FEF72BFA8B
S3150800338805469DF84A3013F0100F17D00696089090
S31508003398002106A8FEF7AEFD044678B9002106A85E
S315080033A8FEF7E0FF034600B90723042B06D01C46A0
S315080033B804E00624DEE70724DCE70025002CC1D153
S315080033C811A8FFF72DF8044600B935B9002CB9D16C
S315080033D80598FFF77FFB0446B4E70022294611A89B
S315080033E8FEF7C9FE0446F1E7CC1400202DE9F041A2
S315080033F882B080460E46174605460024731E9C4230
S3150800340814DA6B46012201A93846FFF793FC009B9C
S31508003418012B0BD19DF804300D2BEFD06A1C2B70AD
S3150800342801340A2B01D01546E8E7154600232B7008
S315080034381CB1404602B0BDE8F0810020FAE710B595
S3150800344894B00446019100230293039303E00134E0
S3150800345801A8FFF7FEFD21780029F8D1029A002A6B
S315080034680CDB6B4604A90198FFF71DFD48B9009BBC
S31508003478029A9A4208D1039814B010BD4FF0FF304B
S31508003488FAE74FF0FF30F7E74FF0FF30F4E70000B0
S315080034987F2816D931B1FF2812D88038094B33F856
S315080034A81000704700237F2B07D8064A32F81320E6
S315080034B8904202D001339BB2F5E78033D8B2704701
S315080034C800207047E86C0008B0F5805F06D2224BEA
S315080034D81A881AB3904221D3F0B406E01F4BF7E7CF
S315080034E82B461A88CAB1904217D31D1D5B88190A3C
S315080034F8DBB29C18A04204DB0029F1D105EB430393
S31508003508EFE7082909D8DFE801F0050A10131619A4
S315080035181C1F2200861A35F81600F0BC7047821A56
S3150800352802F00103C01A80B2F7E7103880B2F4E750
S31508003538203880B2F1E7303880B2EEE71A3880B220
S31508003548EBE7083080B2E8E7503880B2E5E7A0F53F
S31508003558E35080B2E1E700BFE86D0008DC6F0008B9
S3150800356810B4002304E010F8011B0B44DBB2214613
S315080035784C1E0029F7D1136001205DF8044B7047EB
S315080035880022014B5A707047CC160020034BFE22C6
S31508003598DA7018710222A3F844207047CC16002066
S315080035A810B5054C00232370FFF7EAFFFF23E370E5
S315080035B80123A4F8443010BDCC160020064BFF2280
S315080035C8DA7000221A71597859719A71DA711A7271
S315080035D80622A3F844207047CC16002008B5002018
S315080035E8FFF7D4FF08BD0000074BFF22DA70074A29
S315080035F89A6400221A715A719A710722C3F8072029
S315080036080822A3F844207047CC16002098700008B2
S31508003618044BFF22DA7042689A640122A3F8442010
S31508003628704700BFCC16002010B5084CFF23E3707E
S31508003638E21D4168A06CFFF793FF207100236371B0
S31508003648A3710823A4F8443010BD00BFCC16002087
S3150800365808B53120FFF79AFF08BD000038B5084CB1
S31508003668FF23E370002525716571FDF77BFCA071C2
S31508003678E571257265720723A4F8443038BD00BF82
S31508003688CC16002038B5FDF729FDE8B1FFF778FF15
S315080036980F4C01252570FF23E3701023237100239F
S315080036A86371FDF75FFCA071FDF76EFCE071FDF72D
S315080036B86BFCC0F3072020726572A5720823A4F86C
S315080036C84430FDF7BFF838BD1020FFF75FFF38BD57
S315080036D8CC16002038B505464478FDF743FC013872
S315080036E8844210DC0A4C6A78A16C201DFCF7CEFED1
S315080036F8FF23E3706A78A36C1344A3646B780133D9
S31508003708A4F8443038BD2220FFF740FF38BD00BF73
S31508003718CC16002038B504464578FDF723FC013851
S31508003728854211DC61680A4DA9646278281DFCF790
S31508003738ADFEFF23EB706278AB6C1344AB64637819
S315080037480133A5F8443038BD2220FFF71FFF38BDDE
S31508003758CC16002038B505460D4B9C6CFDF702FCC7
S315080037686A1C411E2046FDF771F860B1084CFF2314
S31508003778E370FDF7F7FB0138A36C0344A364012340
S31508003788A4F8443038BD3120FFF700FF38BD00BF24
S31508003798CC16002038B504464578FDF7E3FB023811
S315080037A885420EDC114BFF22DA700122A3F8442069
S315080037B8617851B9FDF75AF890B93120FFF7E6FE56
S315080037C838BD2220FFF7E2FE38BDA21C074B986CCD
S315080037D8FDF73CF828B16178044A936C0B44936466
S315080037E838BD3120FFF7D2FE38BD00BFCC16002001
S315080037F808B54168074B986CFDF72CF830B1054BAE
S31508003808FF22DA700122A3F8442008BD3120FFF709
S31508003818BDFE08BDCC16002008B5FCF719FE034BFB
S31508003828FF22DA700122A3F8442008BDCC1600202E
S3150800383808B589B2FDF774FB08BD0000054B0022E0
S315080038481A709A6483F84320A3F844209A705A7029
S31508003858704700BFCC160020034B1B780BB101201C
S3150800386870470020704700BFCC1600200022024B84
S3150800387883F84320704700BFCC16002008B50378A4
S31508003888FF2B04D0354A1278012A14D008BDFFF751
S31508003898F9FE324B93F84330012B5AD02F4BB3F924
S315080038A844100029F2DD1846012380F84330033016
S315080038B8FFF7BEFFEAE7C93B352B46D8DFE803F032
S315080038C83345454245453F363C39454545454545D1
S315080038D84545454545454545454545454545454582
S315080038E845454545454545454545241E1B21454508
S315080038F84527452A2D30FFF7EDFECAE7FFF70AFFE9
S31508003908C7E7FFF785FEC4E7FFF78EFEC1E7FFF7AF
S315080039186BFEBEE7FFF762FEBBE7FFF74FFEB8E7A9
S31508003928FFF73EFEB5E7FFF715FFB2E7FFF732FFE9
S31508003938AFE7FFF793FEACE7FFF75AFFA9E7FFF7EC
S315080039486BFFA6E7FFF784FEA3E72020FFF71EFE16
S315080039589FE71020FFF71AFEA0E700BFCC16002045
S3150800396808B50121054800F004FA012803D000F03B
S3150800397803F9012008BD002008BD00BF0000024069
S3150800398808B5642000F0C6F808BD08B500F0C8F800
S3150800399808BD000030B583B00446154B1B7843B103
S315080039A8012C1FD04FF40061124800F0E9F903B062
S315080039B830BD0121042000F05BFA4FF40063009340
S315080039C801258DF804508DF8065000238DF8073028
S315080039D802238DF805306946064800F085F9044B38
S315080039E81D70DDE74FF40061024800F0CBF9DEE709
S315080039F818170020000802407047704700B5C7B07E
S31508003A084FF48C720021684602F06EFF6946094831
S31508003A18FFF762FC40B9009B53B19DF8083013F0D4
S31508003A28100F02D1012000E0002047B05DF804FB22
S31508003A380020FAE7B070000800487047B070000820
S31508003A4808B50748002380F828320A220549FFF7EF
S31508003A58B3F818B90122024B83F8282208BD00BF1B
S31508003A681C170020A070000810B50D4B93F82832D3
S31508003A78012B10D0FCF72EFF00F1640440210948F9
S31508003A8800F008FB18B9FCF725FF8442F6D2064869
S31508003A98FFF74CFC10BD0248FFF750FBEAE700BFEA
S31508003AA81C17002000440040B070000808B5054BF4
S31508003AB893F82832012B00D008BD0248FFF73EFBD1
S31508003AC8FAE700BF1C17002010B504460F4B93F8F9
S31508003AD82832012B15D10D49FFF7B1FC002810DA59
S31508003AE80A48002380F82832FFF728FB09E0084827
S31508003AF800F0C8FA8021064800F0CCFA0028F9D068
S31508003B08013421780029F2D110BD00BF1C17002006
S31508003B1800440040014B1880704700BF4819002030
S31508003B2808B5FCF7D7FE104B1B68984211D30F4B04
S31508003B381B787BB901220D4B1A704FF480510C483B
S31508003B4800F020F9FCF7C6FE0A4B1B881844064BFA
S31508003B58186008BD0022054B1A704FF480510448B6
S31508003B6800F00EF9EEE700BF4C1900204A190020AC
S31508003B78000802404819002008B54FF48051024849
S31508003B8800F0FEF808BD00BF00080240054B1B6997
S31508003B98002B00DB7047034B034A5A6002F1883250
S31508003BA85A60F7E7003C024023016745024A136951
S31508003BB843F0004313617047003C0240014BD8604C
S31508003BC8704700BF003C02400E4BDB6813F4803F89
S31508003BD814D10C4BDB6813F0100F01D00520704781
S31508003BE8084BDB6813F0EF0F01D006207047054B2A
S31508003BF8DB6813F0020F03D00720704701207047CF
S31508003C0808207047003C024000B583B008238DF8A9
S31508003C180730FFF7D9FF8DF8070003E0FFF7D4FF51
S31508003C288DF807009DF80730DBB2012BF6D09DF812
S31508003C38070003B05DF804FB70B5064649B10129CB
S31508003C480DD0022902D04FF4407503E04FF40075F1
S31508003C5800E00025FFF7D8FF082803D070BD4FF409
S31508003C688075F7E70F4C236923F4407323612369AA
S31508003C781D432561236923F0F803236123691E433D
S31508003C8846F002062661236943F480332361FFF769
S31508003C98BBFF236923F002032361236923F0F80392
S31508003CA82361DBE7003C024070B505460E46FFF780
S31508003CB8ABFF082800D070BD0A4C236923F440736B
S31508003CC82361236943F400732361236943F00103DD
S31508003CD823612E60FFF798FF236923F00103236108
S31508003CE8E9E700BF003C024000230F2B40D8F0B498
S31508003CF825E084682240826082684C79AC40224379
S31508003D08826044689FB20126BE4024EA06044460DD
S31508003D1844688A79BA4092B222434260C2689CB221
S31508003D2866000324B44022EA0402C260C268CC7959
S31508003D3804FA05F51543C56001330F2B16D8012279
S31508003D489A400C68A243F7D104685D000322AA408A
S31508003D58D2431440046004680E79AE4034430460C4
S31508003D680C79013CE4B2012CD8D8C2E7F0BC7047FC
S31508003D7870470369194201D100207047012070472E
S31508003D88018370474183704730B401F007039B00ED
S31508003D989A40C908083150F821400F2505FA03F357
S31508003DA824EA030340F8213050F821301A4340F832
S31508003DB8212030BC7047000010B4294B9B6803F0DB
S31508003DC80C03042B23D0082B24D013B1254B0360EE
S31508003DD801E0244B0360224CA368C3F3031322496A
S31508003DE8CB5CDAB20368D3404360A268C2F3822286
S31508003DF88A5CD2B223FA02F28260A268C2F342321D
S31508003E088A5CD2B2D340C3605DF8044B7047174B3F
S31508003E180360E0E7124B5A685B6803F03F0312F445
S31508003E28800F12D0114AB2FBF3F20D4B5B68C3F34D
S31508003E38881303FB02F30A4A5268C2F301420132A5
S31508003E485200B3FBF2F30360C5E7064AB2FBF3F286
S31508003E58034B5B68C3F3881303FB02F3EBE700BF66
S31508003E68003802400024F4000400002000127A00FA
S31508003E7829B9054A136B23EA000010637047024AFA
S31508003E88136B1843106370470038024029B9054A6E
S31508003E98536B23EA000050637047024A536B184372
S31508003EA8506370470038024029B9054A136C23EA5B
S31508003EB8000010647047024A136C18431064704770
S31508003EC80038024029B9054A536C23EA00005064B1
S31508003ED87047024A536C18435064704700380240CA
S31508003EE829B9054A136A23EA000010627047024A8C
S31508003EF8136A184310627047003802402DE9F041EA
S31508003F08038803F44153B1F800C0B1F80280B1F848
S31508003F1804E0CF880E894D898C89CA894CEA080C31
S31508003F284EEA0C0E47EA0E073E4335432C43224316
S31508003F3813430380838B9BB223F400639BB283836A
S31508003F480B8A0382BDE8F08131B903889BB223F056
S31508003F5840039BB20380704703889BB243F0400333
S31508003F6803807047808980B270478181704731B96C
S31508003F7803889BB223F400539BB2038070470388D7
S31508003F889BB243F40053038070470389194201D151
S31508003F98002070470120704730B585B004460D46A5
S31508003FA8038A9BB223F44053CA881343038283893E
S31508003FB89BB223F4B05323F00C03898828896A89AD
S31508003FC801430A431343A381A38A9BB223F440738C
S31508003FD8AA891343A3826846FFF7EEFE204B9C4244
S31508003FE828D003F580639C4224D0029BA28912F448
S31508003FF8004F21D103EB830303EB83032968890068
S31508004008B3FBF1F1174BA3FB0123580905016423F8
S3150800401800FB1313A28912F4004F16D11B01323381
S31508004028104AA2FB0323C3F343132B439BB22381F2
S3150800403805B030BD039BD9E703EB830303EB830382
S3150800404829684900B3FBF1F1DCE7D9003231054AA2
S31508004058A2FB0131C1F3421245EA0203E6E700BFB3
S31508004068001001401F85EB5131B983899BB223F4AF
S3150800407800539BB28381704783899BB243F40053EC
S3150800408883817047C1F30801818070478088C0F32F
S31508004098080070470388194201D10020704701209B
S315080040A870470000024A137843F0010313707047FB
S315080040B81400002030B587B0154D00212846FFF7B3
S315080040C843FF0024ADF804404FF48273ADF8063078
S315080040D8ADF80840ADF80A40ADF80C404FF4007347
S315080040E8ADF80E30ADF81040ADF812400723ADF81C
S315080040F8143001A92846FFF701FF21462846FFF78D
S3150800410836FF01212846FFF71FFF07B030BD00BF5D
S315080041180038004070B582B0214D4FF480512846CA
S31508004128FFF72EFE02238DF8053001238DF804309B
S3150800413800248DF807408DF806404FF4004602A97A
S3150800414841F8086D2846FFF7CFFD31462846FFF7A0
S3150800415817FE10E002211348FFF717FF0028F9D0C9
S31508004168FF211048FFF701FF01210E48FFF70DFF51
S315080041780028F9D00134092CECD94FF400430093F0
S3150800418802238DF804308DF8053000228DF80620B4
S315080041988DF8073069460248FFF7A6FD02B070BDDC
S315080041A800040240003800402DE9F04188B001219A
S315080041B80220FFF75DFE01214FF48040FFF774FEE9
S315080041C84FF48058CDF8048002268DF80960012737
S315080041D88DF8087000248DF80B408DF80A40294D93
S315080041E801A92846FFF780FD41462846FFF7C8FD7E
S315080041F805220D212846FFF7C7FD05220E21284668
S31508004208FFF7C2FD05220F212846FFF7BDFD4FF42B
S31508004218604301938DF808608DF809608DF80A40A7
S315080042288DF80B6001A92846FFF75EFDADF80C402E
S315080042384FF48273ADF80E30ADF81040ADF8124061
S31508004248ADF814404FF40073ADF816303023ADF8C6
S315080042581830ADF81A400723ADF81C30A5F5E63531
S3150800426803A92846FFF74AFE21462846FFF77FFE98
S3150800427839462846FFF768FEFFF74CFF08B0BDE841
S31508004288F08100BF0004024008B501460648FFF75A
S315080042986CFE01210448FFF778FE0028F9D0024889
S315080042A8FFF760FEC0B208BD0038004038B5FCF715
S315080042B811FB00F5FA75FF20FFF7E6FF0446FF280D
S315080042C803D0FCF707FB8542F5D8FF2C14BF00205E
S315080042D8012038BD08B54FF480510348FFF750FD53
S315080042E8FF20FFF7D1FF08BD0004024010B54FF4C0
S315080042F880510848FFF746FDFF20FFF7C5FFFFF77F
S31508004308D5FF10B10124204610BD0446FFF7E2FF89
S31508004318F9E700BF0004024038B504460D4610F018
S31508004328800F06D1FFF7D6FFFFF7E0FF50B9FF2049
S3150800433838BD00F07F0400213720FFF7EDFF01287C
S31508004348F6D8EFE744F04000FFF79EFF280EFFF780
S315080043589BFFC5F30740FFF797FFC5F30720FFF74D
S3150800436893FFE8B2FFF790FF94B10120082C11D00B
S31508004378FFF78AFF0C2C0FD00A24FF20FFF784FFCB
S3150800438810F0800FD4D0631E13F0FF04F5D138BDA2
S315080043989520EBE78720EBE7FF20FFF775FFEBE7AC
S315080043A810B50446FF20FFF76FFF207010BDF8B55B
S315080043B805460E46FCF78EFA00F16407FF20FFF75C
S315080043C863FF0446FF2803D1FCF784FA8742F5D829
S315080043D8FE2C01D00020F8BD6C1C2846FFF7E0FF2C
S315080043E820460235FFF7DCFF023EF5D1FF20FFF72E
S315080043F84BFFFF20FFF748FF0120F8BD70B50546BB
S315080044080C46FFF753FF034608B9184670BD204601
S31508004418FFF73AFFFD2C1BD04FF400762C4614F80C
S31508004428020BFFF731FF6878FFF72EFF2546023E95
S31508004438F4D1FF20FFF728FFFF20FFF725FFFF200D
S31508004448FFF722FF00F01F00052803D00023DCE74A
S315080044580123DAE70123D8E7002840F09A80F0B567
S3150800446883B004464C4B1B7813F0020F04D04A4B12
S315080044781878C0B203B0F0BDFFF796FE4FF4805126
S315080044884648FFF77FFC00210846FFF745FF054623
S31508004498012810D0424B1C60FFF71CFF002C75D072
S315080044A83D4A137803F0FE031370FFF703FE3A4BF1
S315080044B81878C0B2DEE7FCF70DFA00F57A764FF4FD
S315080044C8D5710820FFF728FF012846D00021A92022
S315080044D8FFF722FF012854D92F46FCF7FBF9864235
S315080044E805D900212846FFF717FF0028F5D1FCF75C
S315080044F8F1F98642CED94FF400711020FFF70CFF68
S315080045080028C7D13C46C5E7FF20FFF7BDFE02AB2A
S315080045182B4403F8040C0135EDB2032DF4D99DF8A4
S315080045280630012BB6D19DF80730AA2BB2D1FCF775
S31508004538D1F9864206D94FF08041A920FFF7ECFE4B
S315080045480028F4D1FCF7C6F98642A3D900213A20F7
S31508004558FFF7E2FE054658B19CE72546DDE7FF204A
S31508004568FFF792FE02AB2B4403F8040C0135EDB2B3
S31508004578032DF4D99DF8043013F0400F04D00C2409
S3150800458888E70227A925A8E7042483E7FFF78AFD11
S315080045988DE70120704700BF140000200004024080
S315080045A85019002018B9034B1878C0B27047012073
S315080045B8704700BF1400002008B10420704738B5BA
S315080045C80D461C460BB9042038BD1B4B1B7813F047
S315080045D8010F01D0032038BD184B1B6813F0080FCC
S315080045E800D15202012C18D011461220FFF794FE6A
S315080045F868B94FF400712846FFF7D9FE18B105F5D2
S315080046080075013CF5D100210C20FFF785FEFFF760
S3150800461861FE201C18BF012038BD11461120FFF77E
S315080046287BFE0028F3D14FF400712846FFF7BFFE3A
S315080046380028ECD00024EAE71400002050190020CE
S3150800464808B10420704770B50D4616461C460BB9C6
S31508004658042070BD234B1B7813F0010F01D00320EB
S3150800466870BD204B1B7813F0040F01D0022070BDD3
S315080046781D4B1B6813F0080F00D15602012C1BD0DE
S3150800468813F0060F26D131461920FFF745FE68B9FB
S31508004698FC212846FFF7B2FE18B105F50075013C5E
S315080046A8F6D1FD210020FFF7A9FEC0B1FFF712FEDB
S315080046B8201C18BF012070BD31461820FFF72CFEB4
S315080046C80028F3D1FE212846FFF798FE0028EDD0EA
S315080046D80024EBE721469720FFF71EFED3E70124BF
S315080046E8E4E700BF140000205019002030B585B053
S315080046F818B10424204605B030BD924B1B7813F038
S31508004708010F01D00324F5E714460E2900F20B81A0
S31508004718DFE811F00F00160009015F000901090119
S315080047280901090109010901BB00C200D100DF001E
S31508004738F100FFF7DBFD002840F0F7800124A8E028
S3150800474800210920FFF7E8FD08B10124A1E010219E
S315080047586846FFF72CFE002800F0E9809DF800302F
S315080047689B09012B24D09DF8053003F00F039DF80B
S315080047780A2003EBD2139DF80920520002F006021C
S315080047881344DBB20233DBB29DF808109DF8072004
S31508004798920002EB91129DF80610890201F4406115
S315080047A80A440132093B02FA03F32360002470E045
S315080047B89DF809309DF8082003EB02239DF8072089
S315080047C8120402F47C12134401339B02236000246A
S315080047D85FE05D4B1B6813F0040F21D000218D2084
S315080047E8FFF79AFD08B1012453E0FF20FFF74CFDB7
S315080047F810216846FFF7DBFD80B9012449E0FF2050
S31508004808FFF742FD013DEDB2002DF8D19DF80A30BB
S315080048181A0910239340236000243AE03025F3E769
S3150800482800210920FFF778FD08B1012431E010219D
S315080048386846FFF7BCFD00287BD0434B1B6813F07E
S31508004848020F11D09DF80A305B0003F07E039DF82D
S315080048580B2003EBD21301339DF80D209209013A78
S3150800486893402360002414E09DF80A30C3F38402B9
S315080048789DF80B10CB0003F0180303EB5113013313
S3150800488802FB03332360002403E02F4B1B681370D5
S315080048980024FFF71FFD2DE700210920FFF73CFD3F
S315080048A808B10124F5E710212046FFF780FD002806
S315080048B841D10124EDE700210A20FFF72DFD08B1B3
S315080048C80124E6E710212046FFF771FDA8BB01245D
S315080048D8DFE700213A20FFF71FFD054638B1012416
S315080048E8D7E7FF20FFF7D0FC60550135EDB2032D59
S315080048F8F7D90024CDE7144B1B6813F0040F01D130
S315080049080124C6E700218D20FFF706FD08B101241A
S31508004918BFE7FF20FFF7B8FC40212046FFF747FD11
S3150800492868B90124B5E70424B3E70024B1E70124EC
S31508004938AFE70124ADE70024ABE70024A9E7002484
S31508004948A7E700BF140000205019002082B00023F2
S31508004958019300932A4A136843F480331360284B5B
S315080049681B6803F400330093019B01330193009BF2
S315080049781BB9019BB3F5A06FF1D1214B1B6813F442
S31508004988003F06D001230093009B012B04D002B0F8
S31508004998704700230093F7E7194B1A6C42F08052C8
S315080049A81A6418490A6842F440420A609A689A6082
S315080049B89A6842F400429A609A6842F4A0529A6049
S315080049C8114A5A601A6842F080721A600C4B1B68C2
S315080049D813F0007FFAD040F205620C4B1A60A3F573
S315080049E880639A6822F003029A609A6842F0020283
S315080049F89A60034B9B6803F00C03082BF9D1C6E7AA
S31508004A08003802400070004008544007003C024045
S31508004A1810B5104CD4F8883043F47003C4F88830BD
S31508004A280D4B1A6842F001021A60002199601A684B
S31508004A3822F0847222F480321A60084A5A601A6888
S31508004A4822F480221A60D960FFF780FF4FF00063CE
S31508004A58A36010BD00ED00E00038024010300024C5
S31508004A680369024A12685A600020704768190020CC
S31508004A7810B50446D0F8E8351B699847032384F827
S31508004A881231002010BD08B590F8123180F813319C
S31508004A98042380F81231D0F8E835DB6898470020F7
S31508004AA808BD08B5D0F8E435DB6903B19847002096
S31508004AB808BD08B5D0F8E4351B6A9847002008BD34
S31508004AC808B5D0F8E4355B6A9847002008BD10B5E4
S31508004AD80446D0F8E8355B699847012384F8153108
S31508004AE8002010BD10B50446D0F8E8359B699847EC
S31508004AF8D4F8E4355B68002120469847002084F8F6
S31508004B08150110BD10B5044600234022194601F0C8
S31508004B189DF8002340228021204601F097F80123BA
S31508004B2884F81231D4F8E8355B68A07898470020ED
S31508004B3810BD10B582B00446694600F073F99DF8B1
S31508004B48001001F01F03012B0FD03BB1022B11D027
S31508004B5801F08001204601F015F903E06946204670
S31508004B6800F0D1FA002002B010BD6946204600F0D0
S31508004B78EEFAF7E76946204600F006FBF2E710B5B5
S31508004B88044600294CD190F81131022B05D094F827
S31508004B981631012B3DD0002010BDD0F83821D0F8A9
S31508004BA824319A4212D9D21AC0F83821C178012973
S31508004BB806D092B2D4F82811204600F0BAF8E6E7EB
S31508004BC8D0F828110B44C0F82831F2E7D0F83C1180
S31508004BD8B1FBF3F203FB12122AB98B4203D8D0F8B9
S31508004BE8403199420BD3D4F8E435DB681BB194F805
S31508004BF81221032A0AD0204600F0BAF8C7E7114658
S31508004C0800F097F80023C4F84031C0E720469847D3
S31508004C18F1E72046FFF724FF002384F81631BAE7A0
S31508004C280A46D0F8E4355B69002BB4D090F812111F
S31508004C380329B0D111469847ADE710B5044669BBB4
S31508004C4890F81131032B32D1D0F89033D0F87C2361
S31508004C58934215D99B1AC0F89033C178012909D00F
S31508004C689A4228BF1A4692B2D4F88013204600F012
S31508004C7868F81CE0D0F880131144C0F88013EFE7F1
S31508004C88D0F8E4351B691BB190F81221032A03D022
S31508004C98204600F05EF80AE09847F9E70A46D0F891
S31508004CA8E4359B691BB190F81211032901D000203D
S31508004CB810BD11469847FAE7F8B504460D46164654
S31508004CC81F4601F08BFCC4F8E475069BC4F8E83562
S31508004CD8C4F8EC652946204600F06AFFD4F8E8359A
S31508004CE81B689847204601F0CBFCF8BD10B504466A
S31508004CF8D0F8E4351B689847D4F8E8359B68984790
S31508004D08002010BD08B5D0F8E4355B689847002040
S31508004D1808BD10B504461346C4F83C21C4F8382122
S31508004D28022280F811210A46002101F008F800201D
S31508004D3810BD08B513460A46002101F000F8002000
S31508004D4808BD08B513460A46002100F0CAFF002028
S31508004D5808BD10B50446042380F8113100231A4605
S31508004D68194600F0ECFF204600F000FF002010BDB1
S31508004D7810B50446052380F8113100231A4619464A
S31508004D8800F0AFFF204600F0F1FE002010BD00231A
S31508004D9802E00133DBB201300278002AF9D118465D
S31508004DA87047000010B504464B88012B02D0022B29
S31508004DB80AD010BDC0F81831D0F8E4359B68984772
S31508004DC82046FFF7C6FF10BD8B8813F0FF0FF0D1FA
S31508004DD8026952681B0A013B042B07D8DFE803F06F
S31508004DE8030F13171B00012363F306120C4B1A60F3
S31508004DF8012384F816312046FFF7ABFFD9E70223CB
S31508004E0863F30612F2E7032363F30612EEE70423B5
S31508004E1863F30612EAE7052363F30612E6E700BF1B
S31508004E286819002090F8CC350B7090F8CD354B7082
S31508004E3890F8CE3590F8CF2503EB02234B8090F8EF
S31508004E48D03590F8D12503EB02238B8090F8D2351C
S31508004E5890F8D32503EB02239BB2CB80C0F84031E8
S31508004E68012380F81131704710B50446802100F0F7
S31508004E7889FF0021204600F085FF204600F076FECF
S31508004E8810BD30B583B005460C464A88130A013B5F
S31508004E98062B6ED8DFE803F00416296D6D656900E0
S31508004EA8D0F8EC351B680DF1060180789847E38839
S31508004EB8402B03D095F81231012B0ED10823ADF8F3
S31508004EC806300AE0D0F8E4359B6A0DF106018078C9
S31508004ED8984702234370C5F8F005BDF8062012B1B5
S31508004EE8E388002B49D103B030BDD2B2052A34D89D
S31508004EF8DFE802F0030B131B232BD0F8EC355B68AD
S31508004F080DF1060180789847E7E7D0F8EC359B68F5
S31508004F180DF1060180789847DFE7D0F8EC35DB68AD
S31508004F280DF1060180789847D7E7D0F8EC351B6964
S31508004F380DF1060180789847CFE7D0F8EC355B691C
S31508004F480DF1060180789847C7E7D0F8EC359B69D4
S31508004F580DF1060180789847BFE72146FFF784FFD9
S31508004F68C1E72146FFF780FFBDE72146FFF77CFF2B
S31508004F78B9E72146FFF778FFB5E79A4228BF1A46E8
S31508004F88ADF8062001462846FFF7C3FEABE738B555
S31508004F9804468B88E3B9CB88D3B98D7805F07F05A5
S31508004FA890F81231032B0CD080F81451294600F0DA
S31508004FB82BFF2046FFF7CDFE35B1022384F81231C0
S31508004FC838BDFFF751FF38BD012384F8123138BDC3
S31508004FD82046FFF749FF38BD10B504468B78204AA6
S31508004FE81370012B08D890F81221022A07D0032A31
S31508004FF815D0FFF739FF10BDFFF736FF10BD5BB1B7
S3150800500880F81031032280F812211946FFF76EFE40
S315080050182046FFF79EFE10BDFFF79BFE10BD83B125
S3150800502890F810118B4218D0FFF76CFE0C4B1978C4
S3150800503884F810112046FFF759FE2046FFF789FE27
S3150800504810BD022280F8122180F810311946FFF7A0
S3150800505859FE2046FFF77DFE10BDFFF77AFE10BD04
S315080050686019002008B5CB88012B08D190F81231B1
S31508005078022B07D0032B0AD0FFF7F6FE08BDFFF769
S31508005088F3FE08BD01220549FFF743FE08BD0122C4
S3150800509800F58871FFF73DFE08BD00BF58190020C6
S315080050A808B590F81231023B012B0DD80122084B9E
S315080050B81A60D0F8183113B10322054B1A60022278
S315080050C80349FFF726FE08BDFFF7CEFE08BD00BF59
S315080050D85419002010B5044690F81231023B012BEA
S315080050E80ED84B88012B00D010BD0023C0F8183104
S315080050F8D0F8E4359B6898472046FFF72AFE10BD86
S31508005108FFF7B2FEF0E708B54B78092B1CD8DFE89D
S3150800511803F012181B151B09051B0F0CFFF7B1FE28
S31508005128002008BDFFF733FFFAE7FFF755FFF7E753
S31508005138FFF798FFF4E7FFF7B3FFF1E7FFF732FE4B
S31508005148EEE7FFF7C7FFEBE7FFF78EFEE8E738B5A8
S3150800515804460D4690F81231032B11D10B79012B11
S3150800516803D9FFF781FE002038BDD0F8E4359B68DF
S315080051789847EB88002BF6D12046FFF7EAFDF2E7B9
S31508005188FFF772FEEFE7000038B505460C468A8831
S31508005198D1B26378012B25D0002B46D0032B1FD11B
S315080051A890F81231022B05D0032B09D02146FFF7B8
S315080051B85BFE15E0A1B1802912D000F0E3FD0FE0EF
S315080051C8638823B919B1802901D000F0DBFDD5F829
S315080051D8E4359B682146284698472846FFF7B9FDCF
S315080051E8002038BD90F81231022B05D0032B0AD0BF
S315080051F82146FFF739FEF3E70029F1D08029EFD0D9
S3150800520800F0C0FDECE76388002BE9D149B1802995
S3150800521807D000F0D8FDD5F8E4359B68214628461E
S3150800522898472846FFF795FDDAE790F81231022BDA
S3150800523805D0032B0AD02146FFF716FED0E700292A
S31508005248CED08029CCD000F09DFDC9E712F0800F9A
S315080052580FD101EB8101CB00034493F87633CBB128
S3150800526801220E4B1A6002220C492846FFF751FD07
S31508005278B6E701F07F0101EB8101CB00034493F8FF
S315080052881E311BB10122054B1A60ECE70022034BBD
S315080052981A60E8E70022014B1A60E4E75C19002067
S315080052A8D0B170B50D4616460446FFF770FD0130B5
S315080052B8400080B23080287003236B70022307E011
S315080052C85A1CD2B20134E9540233DBB20021A9547C
S315080052D821780029F4D170BD70470000C3684FF0E3
S315080052E8FF325A60C3686FF080425A61014BC26840
S315080052F8936170470008008030B583B005460024DE
S315080053080194032001F0BDF9EB681A69019201348A
S315080053180E4A944217D8019A002AF2DA019A42F0FC
S3150800532801020192019A1A610023EA681269019238
S315080053380133064A934203D8019A12F0010FF4D1B1
S31508005348032001F09EF9002003B030BD400D03008C
S3150800535810B4C4786CB903339C10323200EB82005F
S315080053688068002303E051F8042B02600133A34246
S31508005378F9D300205DF8044B704710B40332921035
S31508005388D0F8D040002303E0206841F8040B013325
S315080053989342F9D308465DF8044B704730B40023A6
S315080053A8C3700123837040238380012910D0E9B98B
S315080053B80023C3720C230370062343704FF4A063BB
S315080053C8C3802A4CC46004F50063036100231FE008
S315080053D80123C37208230370042343704FF4A07390
S315080053E8C380022303724FF0A044EBE70024E9E7E1
S315080053F804EB431202F51065191D00EB81018D6057
S3150800540802F5306203F1140100EB81014A600133A9
S3150800541842789342ECD304F58063436104F58863C4
S31508005428C0F8CC30002309E004EB431101F5A0616C
S3150800543803F1220200EB8202916001330578AB4240
S31508005448F2D3002309E004EB033101F5805103F197
S31508005458320200EB820291600133AB42F3D304F5C2
S315080054686064C0F80C41002030BC70470000044056
S3150800547838B50446037A012B16D0C268D16841F0BC
S315080054884003D360FFF738FF4FF45023627A0AB116
S315080054984FF4E813E2689363142001F0FDF8E37803
S315080054A8012B24D0002038BD0025C268936B6FF302
S315080054B81043417A09B143F480139363E268D368C9
S315080054C86FF386136FF396536FF351436FF3D34312
S315080054D8D3602046FFF710FFE378012BDFD10523B9
S315080054E863F3440545F02005E3689D60D7E7E3685C
S315080054F89D68052262F3440545F020059D60D1E7BD
S31508005508C268936843F00103936000207047C26835
S31508005518936823F0010393600020704700B583B0B1
S3150800552800230193019A42F020020192019A61F33D
S315080055388A120192C26801991161C26812690192B8
S315080055480133074A934203D8019A12F0200FF4D17F
S31508005558032001F096F8002003B05DF804FB00BFAD
S31508005568400D030000B583B000230193019A42F069
S3150800557810020192C26801991161C2681269019202
S315080055880133074A934203D8019A12F0100FF4D14F
S31508005598032001F076F8002003B05DF804FB00BF8D
S315080055A8400D030008B5C268D3686FF35D736FF3DF
S315080055B89E73012908D009B943F08043D360322085
S315080055C801F06AF8002008BD43F00053F6E7C368FF
S315080055D8586900F00100704708B5FFF7F8FF10F1A1
S315080055E8FF3018BF012008BDC36858699B69184071
S315080055F870470269136861F301031360704738B589
S3150800560805460024C3689C61C3686FF080425A61E6
S31508005618FFF764FEEB7803B9102444F0804444F499
S31508005628701444F4605444F00C04EA68936923EA55
S3150800563804031C439461002038BD70B50446002550
S31508005648D0F80C311D600269136865F3CC23136022
S31508005658C37A012B12D010212046FFF75FFF204698
S31508005668FFF780FF236900221A6123695A612369B3
S315080056784FF0FF3199612369DA6136E02E46032136
S31508005688FFF7B7FFE26880235362202262F31F45BB
S3150800569863F30F05E1688D62A02161F30F0663F3D2
S315080056A81F46E368C3F804614FF4907363F30F0663
S315080056B862F31F46E368C3F808614FF4A07363F3FF
S315080056C80F066FF31F46E368C3F80C61C3E74FF08C
S315080056D89041131D04EB83039868016099680020BC
S315080056E808619B68FF219960013263789A4208D25B
S315080056F8131D04EB83039B681B68002BE7DB00215B
S31508005708E7E700220EE04FF0904102F1140304EB9C
S315080057188303586801605968002008615B68FF219F
S315080057289960013263789A4209D202F1140304EBAC
S3150800573883035B681B68002BE5DB0021E5E7226924
S31508005748136943F480731361E378012B04D0204668
S31508005758FFF755FF002070BD0323402262F38A0332
S3150800576843F4803362F3594322691363EFE7036905
S315080057789B68C3F34103022B04D005D8012B03D039
S3150800578803207047012070470220704703699B6809
S3150800579882691168C3F34103022B0AD1032363F311
S315080057A80A0111600269536843F480735360002044
S315080057B870476FF30A01F4E730B400244B78012BDD
S315080057C822D00D7805F1140200EB820252680123F3
S315080057D8AB4063F31F44136813F4004F0DD18D686B
S315080057E865F30A03CD7865F39343897961F3995389
S315080057F843F0805343F4004313600269D369234393
S31508005808D361002030BC70470D782A1D00EB820250
S315080058189268AB4063F30F04DDE770B400221546BF
S315080058284B78012B14D00B7803F1140400EB84048D
S3150800583864680121994061F31F456FF3CF322260EE
S315080058480269D36923EA0503D361002070BC70474F
S315080058580E78311D00EB81018C68B34063F30F05A0
S31508005868EBE738B54B78012B25D00B78143300EBCA
S3150800587883035B681A681C694B69002B74D18B68AB
S3150800588863F31204012363F3DC440B78143300EB47
S3150800589883035B681C61C378012B73D0CB78012B13
S315080058A878D042F004420B78143300EB830043683F
S315080058B81A60002038BD0B78043300EB83039B6815
S315080058C81A681C694B69D3B96FF31204012363F389
S315080058D8DC440B78043300EB83039B681C61C378AC
S315080058E8012B1BD0CB78012B1FD04B69EBB10C7859
S315080058F80123A3400469656B2B43636315E063F3CF
S3150800590812048D682B44013BB3FBF5F363F3DC44BF
S31508005918CB78012BDDD163F35E74DAE70B780433B1
S3150800592800EB83039B680C695C61CB78012B10D06C
S3150800593842F004420B78043300EB83039B681A6031
S31508005948CB78012BB5D18B8A0A78C968FFF700FD91
S31508005958AFE703699B6813F4807F02D142F00052CF
S31508005968E6E742F08052E3E78D682B44013BB3FB38
S31508005978F5F3C3F3090363F3DC4403FB05F363F3A5
S31508005988120482E70B78143300EB83035B680C690F
S315080059985C6183E74B7913B142F0005281E742F024
S315080059A880527EE730B482B04B78012B2ED00B7824
S315080059B8143300EB83035B681A681B6900934B6909
S315080059C8002B6DD18C689DF8003064F306038DF8BA
S315080059D800309DF80230012464F3C4038DF80230C0
S315080059E80B78143300EB83035B68009C1C61C3784F
S315080059F8012B65D042F004420B78143300EB830080
S31508005A0843681A60002002B030BC704783691A6878
S31508005A181C6900944C6914BB9DF800406FF3060492
S31508005A288DF800409DF80240012565F3C4048DF8F9
S31508005A380240009C1C61C478012C29D042F004421B
S31508005A481A60C378002BDDD14B69002BDAD00A78A7
S31508005A58012393400269516B0B435363D2E78D6860
S31508005A68AC420ED94D619DF8004065F306048DF8E1
S31508005A7800409DF80240012565F3C4048DF80240EC
S31508005A88D7E79DF8005064F306058DF80050F0E74F
S31508005A980C78043400EB8404A4680D696561CDE7C5
S31508005AA88C684C619DF8003064F306038DF8003065
S31508005AB89DF80230012464F3C4038DF802308FE799
S31508005AC80B78143300EB83035B680C695C6191E718
S31508005AD84B78012B0AD00B78143300EB8300426805
S31508005AE8116841F400131360002070470B780433DB
S31508005AF800EB830082681368002B03DB43F400136A
S31508005B081360F1E743F08043F8E74B78012B0FD091
S31508005B180B78143300EB8300406802686FF355521C
S31508005B28CB78023BDBB2012B08D90260002070470C
S31508005B380B78043300EB83008068EEE742F0805266
S31508005B48F3E703699869DB691840000C7047143154
S31508005B5800EB81014B689A680369586910407047D9
S31508005B6803699869DB69184080B2704782B00023D8
S31508005B780093C0238DF803304FF00003012262F327
S31508005B88C4038DF8023018238DF80030436D009A47
S31508005B981A61C378012B01D002B07047436D00F231
S31508005BA8CC525A61436D1A684FF080221A60F3E79F
S31508005BB838B50446FFF7F2FB012384F812310022B0
S31508005BC884F8142115E091001144CB0023440121DF
S31508005BD883F81D1183F81C21A3F82221002183F8D4
S31508005BE81F114020C3F82401C3F82811C3F830113F
S31508005BF8013260788242E6D3002214E0910011440B
S31508005C08CB002344002183F8751383F87423A3F87B
S31508005C187A2383F877134025C3F87C53C3F880138F
S31508005C28C3F8881301328242E8D32046FFF76FFC8F
S31508005C382046FFF71DFC00212046FFF7B3FC204647
S31508005C48FFF7FBFC2046FFF75BFC38BD70B54DB285
S31508005C58002D18DB01F07F0606EB8606F40004F52E
S31508005C685C740444043401F07F012170ED0F6570FB
S31508005C78A260E37005B1E180022B0ED02146FFF73A
S31508005C889BFD002070BD01F07F0606EB8606F40032
S31508005C9804F58C7404440434E5E700232371EDE71E
S31508005CA810B54AB2002A12DB01F07F0404EB84041B
S31508005CB8E30003F55C730344043301F07F011970AC
S31508005CC8D20F5A701946FFF7A8FD002010BD01F03B
S31508005CD87F0404EB8404E30003F58C73034404335C
S31508005CE8EBE770B501F07F04A6003519E9000D4603
S31508005CF801F55C71014404312E460544C5F8802334
S31508005D08C5F888330023C5F88C3385F8753385F8C4
S31508005D187443C378012B0AD004EB8404E3000344D4
S31508005D2893F8743343B1FFF79CFD002070BD3346E2
S31508005D380344C3F88423EFE7FFF734FEF5E770B5A5
S31508005D4801F07F05AE007119CC0004F58C74044483
S31508005D58211D2E44F4000444012684F81D6184F8A4
S31508005D681C51C4F82821C4F82C210022C4F834216F
S31508005D78C4F830311DB1FFF774FD002070BDFFF778
S31508005D8811FEFAE710B54AB2002A12DB01EB8104C4
S31508005D98E30003F55C730344043301249C7001F0A3
S31508005DA87F011970D20F5A701946FFF791FE002025
S31508005DB810BD01F07F0404EB8404E30003F58C733B
S31508005DC803440433E9E710B54AB2002A12DB01EBAB
S31508005DD88104E30003F55C730344043300249C70D0
S31508005DE801F07F011970D20F5A701946FFF78DFE18
S31508005DF8204610BD01F07F0404EB8404E30003F594
S31508005E088C7303440433E9E710B4002461F30A14D5
S31508005E1802691368234313605DF8044B704708B595
S31508005E280369596841F002025A60032000F034FCFD
S31508005E3808BD000010B50446044B1B685B6A984702
S31508005E484FF08043E2685361012010BD44000020EA
S31508005E5838B50446C3685D6815F0040F03D1E368CE
S31508005E685D60012038BD024B1B689B6A9847F6E7B8
S31508005E784400002010B50446837A43B1D0F80C31A3
S31508005E886FF341036FF30003D0F80C2113602269FE
S31508005E98536823F001035360054B1B689B6920462A
S31508005EA898474FF00043E2685361012010BD00BFD0
S31508005EB84400002030B583B0054600248DF8074015
S31508005EC890F812318DF80730164B1B685B699847AE
S31508005ED82B699A684FF40064EB685C61AB7A33B156
S31508005EE812F0010F03D095F81531012B02D00120C5
S31508005EF803B030BD9DF80730DBB2032BF7D1D5F8D0
S31508005F080C21136843F001031360D5F80C211368B4
S31508005F1843F003031360044A136943F00603136145
S31508005F28E5E700BF4400002000ED00E010B5044690
S31508005F38044B1B68DB6898470823E268536101200D
S31508005F4810BD00BF4400002010B50446044B1B686A
S31508005F58DB6998474FF48013E2685361012010BD46
S31508005F684400002010B50446044B1B681B6A984772
S31508005F784FF40013E2685361012010BD4400002065
S31508005F8803691A695B6BCB40DB01DBB21343043147
S31508005F9800EB810082689068184070472DE9F04147
S31508005FA80746FFF7CEFD0446002520E005F1140351
S31508005FB807EB83035B681969AA002A44D3003B44A4
S31508005FC8D3F87C23C1F31201521AC3F88C2327E0AD
S31508005FD816F0020F06D0022605F1140307EB830311
S31508005FE85B689E6016F0080F2DD101356408002CF1
S31508005FF836D014F0010FF8D05FFA85F841463846CE
S31508006008FFF7A5FD064610F0010FE1D0012605F1B8
S31508006018140307EB83035B689E60FB78B342C5D01D
S31508006028114B1B681B68414638469847FB78012B75
S31508006038CED1002DCCD197F81131052BC8D13846C9
S31508006048FFF794FDC4E7084B1B689B6838469847D2
S31508006058082605F1140307EB83035B689E60C4E70B
S315080060680120BDE8F08100BF440000202DE9F04179
S3150800607807460D468A000A44D3000344D3F830215C
S31508006088D3F83411521AD3F824319A4200D8134651
S3150800609803F103084FEA98082B1D07EB83039B684F
S315080060A89B691DE006F103084FEA9808AB002B44E4
S315080060B8DC003C44B3B2EAB2D4F828113846FFF7F4
S315080060C847F9D4F828313344C4F82831D4F8343198
S315080060D81E44C4F834612B1D07EB83039B689B6930
S315080060E89BB2984515D2AB002B44DA003A44D2F84D
S315080060F83411D2F8303199420BD253B15B1A05EBF9
S315080061088501CA003A44D2F82461B342CAD81E4661
S31508006118C8E70120BDE8F0812DE9F0410746FFF7F9
S315080061281FFD0446002624E0012303FA06F0396910
S315080061384A6B22EA00024A631D46321D07EB8202B1
S31508006148926893602C4B1B685B68414638469847AB
S31508006158FB78AB421CD1DEB997F81131042B17D15D
S315080061683846FFF703FD13E015F0800F35D10136E1
S315080061786408002C3CD014F0010FF8D05FFA86F8B2
S3150800618841463846FFF7FCFE054610F0010FCBD10D
S3150800619815F0080F05D00825331D07EB83039B6800
S315080061A89D6015F0100F05D01025331D07EB8303E6
S315080061B89B689D6015F0400F05D04025331D07EBF9
S315080061C883039B689D6015F0020FCDD00225331D09
S315080061D807EB83039B689D60C6E731463846FFF799
S315080061E845FF8025331D07EB83039B689D60BEE743
S315080061F80120BDE8F08100BF440000202DE9F041E8
S315080062080446C268936923F010039361C3681D6A3C
S3150800621805F00F06C5F34343022B09D0062B23D0F6
S31508006228E268936943F0100393610120BDE8F081A1
S3150800623847F6F0732B42F3D0C5F30A154FEA8608DA
S3150800624808EB0603DF0007442A46D7F88013FFF74A
S3150800625894F8D7F880332B44C7F88033D7F88C33AB
S315080062681D44C7F88C53DBE7082200F2CC51FFF728
S3150800627884F8C5F30A15B3009919CA002244D2F856
S315080062888C331D44C2F88C53CAE700002DE9F8433D
S3150800629804460025A8462F462E460269536823F069
S315080062A8010353602946FFF739F92B460CE01A1DF6
S315080062B804EB82029268FF21916003F1140204EB51
S315080062C8820252689160013362789342EFD3236958
S315080062D84FF0FF329A614FF0010969F30F0569F328
S315080062E81F452369DD6148F00B082369C3F8148044
S315080062F847F00B0723691F61226913686FF30A13AE
S3150800630813602046FFF732FC46F48056E3685E6160
S31508006318034B1B681B69204698474846BDE8F8831F
S315080063284400002038B50446FFF730FAE368DD680C
S315080063382046FFF71CFA03280ED00123A370402332
S31508006348A380052363F38D25E368DD604FF40053C6
S31508006358E2685361012038BD0023A3704FF4007327
S31508006368A380092363F38D25EEE72DE9F84305464F
S31508006378FFF732F918B900242046BDE8F8832846FD
S31508006388FFF732F9044606460028F5D0C0F3074851
S3150800639818F0080F33D1002418F0040F34D1F7B2D7
S315080063A817F0020F02D00223EA685361C6F307639F
S315080063B85FFA83F913F0800F2BD1C6F3072616F078
S315080063C8080F2BD117F0080F2DD117F0100F2FD162
S315080063D816F0100F31D116F0200F33D118F0100F20
S315080063E835D118F0200F37D119F0400F39D117F0E9
S315080063F8040FC1D02846FFF72BFD0443BCE72846FF
S31508006408FFF7CCFD0446C7E72846FFF785FE044391
S31508006418C5E72846FFF72EFD0443CEE72846FFF7CB
S3150800642849FD0443CEE72846FFF780FD0443CCE739
S315080064382846FFF7E3FE0443CAE72846FFF726FF80
S315080064480443C8E72846FFF76DFF0443C6E728460E
S31508006458FFF77AFD0443C4E72846FFF783FD04439C
S31508006468C2E72846FFF7E6FC0443C0E72DE9F043F0
S3150800647883B001210846FDF7FBFC01240094002699
S315080064888DF804608DF8076002258DF80550384F99
S3150800649869463846FDF728FC21464FF40030FDF7D3
S315080064A803FD21462046FDF7E3FC07222946384620
S315080064B8FDF76AFC072203213846FDF765FC8DF8C7
S315080064C806608DF807408DF804504FF00408CDF89B
S315080064D800808DF8055069463846FDF705FC8DF8A5
S315080064E804504FF00809CDF8009069463846FDF77C
S315080064F8FBFB21462846FDF7BBFC07F58067092202
S3150800650849463846FDF740FC092211463846FDF744
S315080065183BFC4FF4407300938DF804508DF80550F2
S315080065288DF806608DF8074069463846FDF7DCFBA6
S3150800653821464FF00070FDF7B7FC21464046FDF7A7
S3150800654897FC4FF4805700978DF804408DF806603D
S315080065588DF807408DF80550064C69462046FDF724
S31508006568C3FB39462046FDF70BFC03B0BDE8F083AC
S31508006578000002400008024008B5FFF777FFFAF75F
S3150800658871FCFAF77FFCFCE7DFF834D0002103E05A
S315080065980C4B5B58435004310B480C4B42189A4233
S315080065A8F6D30B4A02E0002342F8043B094B9A4209
S315080065B8F9D3FEF72DFA00F053F9FFF7DDFF704718
S315080065C8000002203872000800000020B4020020EB
S315080065D8B4020020AC1A0020FEE7000070B582B0AD
S315080065E801210846FDF744FC4FF4C05300930326DF
S315080065F88DF8056002238DF8043000258DF80650BD
S315080066088DF807501D4C69462046FDF76DFB0A2292
S315080066180B212046FDF7B8FB0A220C212046FDF778
S31508006628B3FB01210420FDF723FC4FF40063009314
S3150800663801248DF804408DF806508DF807408DF82A
S31508006648056005F1804505F5023569462846FDF7D2
S315080066584BFB6B6923F400636B6121464FF480405A
S31508006668FDF730FC21468020FDF710FC21464FF047
S315080066788050FDF735FC02B070BD00BF000002402F
S31508006688704704E000BF01331B2BFBD91046421E96
S3150800669808B10023F8E7704708B54FF47A7303FB87
S315080066A800F0FFF7EEFF08BD20230B80004870476F
S315080066B87400002008B590F81231032B01D0002089
S315080066C808BDFAF735FBFAE708B5FAF731FB0020F3
S315080066D808BD08B50846FAF75FFB002008BD0000A4
S315080066E808B50B7813F0600F06D14B780A2B14D02F
S315080066F80B2B17D0062B01D0002008BD4B881B0A88
S31508006708212B04D00B491722FEF703FBF4E7CA88A6
S31508006718172A28BF17220849F6E701220749FEF76C
S31508006728F8FAE9E78B7813B9044A1360E4E7FEF741
S315080067389BFBE1E77D000020860000206419002005
S3150800674810B504468121FFF7ABFA01212046FFF769
S31508006758A7FA002010BD000010B5044602234022FF
S315080067688121FFF773FA0223402201212046FFF709
S315080067786DFA4023034A01212046FFF7B2FA0020A2
S3150800678810BD00BF6C1A0020004870476C1A00201C
S3150800679812230B80004870479400002004230B80BE
S315080067A800487047A800002010B5044C0A46214640
S315080067B80348FEF775FD204610BD00BF6C1900207A
S315080067C80071000810B5044C0A4621460348FEF72E
S315080067D867FD204610BD00BF6C190020F070000840
S315080067E810B5044C0A4621460348FEF759FD2046CB
S315080067F810BD00BF6C1900201471000810B5044CB0
S315080068080A4621460348FEF74BFD204610BD00BF41
S315080068186C190020D070000810B5044C0A462146A9
S315080068280348FEF73DFD204610BD00BF6C19002041
S31508006838D870000870477047704708B5FDF7DCF848
S3150800684808BD08B5FDF7D9F808BD08B50120FDF754
S31508006858A1F808BD08B50020FDF79CF808BD00009A
S3150800686870B50D4E0D4CA41BA4100025A54209D1E0
S315080068780B4E0C4C00F04EF8A41BA4100025A5429C
S3150800688805D170BD56F8253098470135EEE756F814
S31508006898253098470135F2E730720008307200084B
S315080068A83072000834720008044B054A1B681B6AD4
S315080068B8002B08BF1346D3F8EC0070475002002097
S315080068C8E400002082B001B901A942B14BB113789E
S315080068D80B601278101C18BF012002B070471046CA
S315080068E8FBE76FF00100F8E702440346934200D13C
S315080068F8704703F8011BF9E749B1FF2A85BF8A23C0
S3150800690803600A704FF0FF3098BF012070470846A9
S3150800691870470000F8B500BFF8BC08BC9E4670472B
S31108006928F8B500BFF8BC08BC9E467047D6
S315080069342E2E2F2E2E2F2E2E2F2E2E2F536F757270
S3150800694463652F41524D434D345F53544D3332469C
S31508006954342F63616E2E63000502060206030703DD
S315080069640803090309040A040B040C040C050D05A1
S315080069740E050F050F0610061007100800800008FC
S31508006984004000000200000000C0000800400000AB
S3150800699403000000000001080000010004000000D4
S315080069A400000208000002000500000000000408B8
S315080069B400000200060000000000060800000200AD
S315080069C40700000000000808000002000800000094
S315080069D400000A08000002000900000000000C0874
S315080069E4000002000A00000000000E080000020071
S315080069F40B00000000000800100018002000280002
S31508006A0430003800400048005000580080008800D4
S31508006A1490009800A000A800B000B800C000C80004
S31508006A24D000D8002E2E2F2E2E2F2E2E2F2E2E2F80
S31508006A34536F757263652F41524D434D345F5354FA
S31508006A444D333246342F756172742E63000000008C
S31508006A542E2E2F2E2E2F2E2E2F2E2E2F536F75724F
S31508006A6463652F41524D434D345F53544D3332467B
S31508006A74342F7573622E6300303A00002E2E2F2EA3
S31508006A842E2F2E2E2F2E2E2F536F757263652F667B
S31508006A94696C652E630000004669726D77617265DC
S31508006AA420757064617465207265717565737420E8
S31508006AB464657465637465640A0D00004F70656ED9
S31508006AC4696E67206669726D776172652066696C9E
S31508006AD46520666F722072656164696E672E2E2E54
S31508006AE4000000004552524F520A0D004F4B0A0D42
S31508006AF4000000005374617274696E6720746865D7
S31508006B042070726F6772616D6D696E672073657147
S31508006B1475656E63650A0D0050617273696E672048
S31508006B246669726D776172652066696C6520746F33
S31508006B342064657465637420657261736520626C8C
S31508006B446F636B732E2E2E0045726173696E672010
S31508006B54000000002062797465732066726F6D20E8
S31508006B646D656D6F727920617420307800000000BD
S31508006B7452656164696E67206C696E652066726F1A
S31508006B846D2066696C652E2E2E4552524F520A0D9B
S31508006B9400000000496E76616C6964206368656369
S31508006BA46B73756D20666F756E642E2E2E45525264
S31508006BB44F520A0D0000000050726F6772616D6DC6
S31508006BC4696E67200000000020627974657320747A
S31508006BD46F206D656D6F72792061742030780000BE
S31508006BE457726974696E672070726F6772616D2077
S31508006BF4636865636B73756D2E2E2E00436C6F7315
S31508006C04696E67206669726D776172652066696C5C
S31508006C14650A0D004669726D776172652075706440
S31508006C24617465207375636365737366756C6C79D3
S31508006C3420636F6D706C657465640A0D000000004E
S31508006C44809A45418E418F804545454949498E8FED
S31508006C549092924F994F555559999A9B9C9D9E9FF0
S31508006C6441494F55A5A5A6A7A8A9AAABACADAEAFF1
S31508006C74B0B1B2B3B4B5B6B7B8B9BABBBCBDBEBF8A
S31508006C84C0C1C2C3C4C5C6C7C8C9CACBCCCDCECF7A
S31508006C94D0D1D2D3D4D5D6D7D8D9DADBDCDDDEDF6A
S31508006CA4E0E1E2E3E4E5E6E7E8E9EAEBECEDEEEF5A
S31508006CB4F0F1F2F3F4F5F6F7F8F9FAFBFCFDFEFF4A
S31508006CC401030507090E10121416181C1E000000ED
S31508006CD4222A3A3C3E3F7C7F000000002B2C3B3D99
S31508006CE45B5D0000C700FC00E900E200E400E00088
S31508006CF4E500E700EA00EB00E800EF00EE00EC0030
S31508006D04C400C500C900E600C600F400F600F20097
S31508006D14FB00F900FF00D600DC00A200A300A500D2
S31508006D24A7209201E100ED00F300FA00F100D1007A
S31508006D34AA00BA00BF001023AC00BD00BC00A10025
S31508006D44AB00BB00912592259325022524256125B0
S31508006D546225562555256325512557255D255C2528
S31508006D645B251025142534252C251C2500253C25B2
S31508006D745E255F255A2554256925662560255025EF
S31508006D846C256725682564256525592558255225C2
S31508006D9453256B256A2518250C25882584258C25D5
S31508006DA490258025B103DF009303C003A303C3031F
S31508006DB4B500C403A6039803A903B4031E22C60395
S31508006DC4B50329226122B1006522642220232123E6
S31508006DD4F7004822B0001922B7001A227F20B20011
S31508006DE4A025A00061001A03E0001703F8000703B2
S31508006DF4FF00010078010001300132010601390162
S31508006E0410014A012E017901060180014D00430251
S31508006E148101820182018401840186018701870137
S31508006E2489018A018B018B018D018E018F019001E5
S31508006E349101910193019401F60196019701980134
S31508006E4498013D029B019C019D0120029F01A0011E
S31508006E54A001A201A201A401A401A601A701A701F8
S31508006E64A901AA01AB01AC01AC01AE01AF01AF01A6
S31508006E74B101B201B301B301B501B501B701B80156
S31508006E84B801BA01BB01BC01BC01BE01F701C001CE
S31508006E94C101C201C301C401C501C401C701C801B6
S31508006EA4C701CA01CB01CA01CD011001DD010100E8
S31508006EB48E01DE011201F3010300F101F401F4016C
S31508006EC4F8012801220212013A020900652C3B0244
S31508006ED43B023D02662C3F02400241024102460241
S31508006EE40A015302400081018601550289018A017B
S31508006EF458028F015A0290015C025D025E025F022B
S31508006F0493016102620294016402650266026702E1
S31508006F14970196016A02622C6C026D026E029C014C
S31508006F24700271029D01730274029F017602770250
S31508006F34780279027A027B027C02642C7E027F0242
S31508006F44A60181028202A9018402850286028702B9
S31508006F54AE014402B101B20145028D028E028F02CE
S31508006F6490029102B7017B030300FD03FE03FF03AE
S31508006F74AC0304008603880389038A03B103110357
S31508006F84C2030200A303A303C4030803CC03030038
S31508006F948C038E038F03D8031801F2030A00F9033E
S31508006FA4F303F403F503F603F703F703F903FA0304
S31508006FB4FA033004200350041007600422018A04EB
S31508006FC43601C1040E01CF040100C004D0044401F3
S31508006FD461052604000000007D1D0100632C001EC7
S31508006FE49601A01E5A01001F0806101F0606201F38
S31508006FF40806301F0806401F0606511F0700591FBA
S31508007004521F5B1F541F5D1F561F5F1F601F080614
S31508007014701F0E00BA1FBB1FC81FC91FCA1FCB1F6C
S31508007024DA1FDB1FF81FF91FEA1FEB1FFA1FFB1FE6
S31508007034801F0806901F0806A01F0806B01F040034
S31508007044B81FB91FB21FBC1FCC1F0100C31FD01F16
S315080070540206E01F0206E51F0100EC1FF21F0100ED
S31508007064FC1F4E21010032217021100284210100E7
S315080070748321D0241A05302C2F04602C0201672C96
S315080070840601752C0201802C6401002D260841FF97
S315080070941A0300004F70656E424C54002F626F6FDE
S315080070A4746C6F672E747874000000002F64656D25
S315080070B46F70726F675F6F6C696D65785F73746DF7
S315080070C43332703430352E737265630044656661F5
S315080070D4756C740057696E5553422042756C6B2063
S315080070E4496E746572666163650000004F70656E6B
S315080070F4424C5420557365720000000057696E555A
S3150800710453422042756C6B204465766963650000BA
S315080071143030303030303030303530430000000005
S315080071244300504F534958002E00002020202020A9
S315080071342020202028282828282020202020202015
S315080071442020202020202020202020881010101005
S315080071541010101010101010101010040404040459
S315080071640404040404101010101010104141414185
S31508007174414101010101010101010101010101016D
S31508007184010101010101101010101010424242427F
S31508007194424202020202020202020202020202023D
S315080071A40202020202021010101020000000000061
S315080071B400000000000000000000000000000000BD
S315080071C400000000000000000000000000000000AD
S315080071D4000000000000000000000000000000009D
S315080071E4000000000000000000000000000000008D
S315080071F4000000000000000000000000000000007D
S31508007204000000000000000000000000000000006C
S31508007214000000000000000000000000000000005C
S3110800722400000000000000000000000050
S30908007230AD01000896
S3090800723489010008B6
S315080072380400000000000000010203040102030420
S315080072480607080901000000434C0008874B000898
S315080072583B4B0008AB4A00080D4B00088F4A00084C
S31508007268794A0008BB4A0008C94A0008D74A0008EC
S31508007278ED4A0008180000206167000849670008F9
S31508007288E96600080000000000000000D166000852
S31508007298DB660008BD660008000000000000000064
S315080072A8B166000809022000010100C0320904007D
S315080072B80002FF000000070581024000FF070501DC
S315080072C8024000FF1201100100000040501DAC608A
S315080072D80001010203010000040309049967000874
S315080072E8A5670008CD670008B1670008E9670008C0
S315080072F805680008216800083D6800083F68000816
S3150800730841680008436800084B6800085368000885
S315080073185D68000843000000000000000000000047
S315080073280000000000000000000000000000000047
S3150800733800000000430000000000000000000000F4
S315080073480000000000000000000000000000000027
S3150800735800000000430000000000000000000000D4
S315080073680000000000000000000000000000000007
S3150800737800000000430000000000000000000000B4
S3150800738800000000000000000000000000000000E7
S315080073980000000043000000000000000000000094
S315080073A800000000000000000000000000000000C7
S315080073B80000000043000000000000000000000074
S315080073C800000000000000000000000000000000A7
S315080073D80000000043000000000000000000000054
S315080073E80000000000000000000000000000000087
S315080073F80000000001690008CD68000800000000C8
S315080074082E7100082C7100082D7100082D710008CE
S315080074182D7100082D7100082D7100082D710008BE
S315080074282D7100082D7100082D710008FFFFFFFF58
S31508007438FFFFFFFFFFFFFFFFFFFF000001004153AB
S315080074484349490000000000000000000000000051
S315080074580000000000000000000000000000415382
S315080074684349490000000000000000000000000031
S3150800747800000000000000000000000000000000F6
S315080074885402002000000000000000000000000070
S3150800749800000000000000000000000000000000D6
S315080074A800000000000000000000000000000000C6
S315080074B800000000000000000000000000000000B6
S315080074C800000000000000000000000000000000A6
S315080074D80000000000000000000000000000000096
S309080074E80000000092
S70508006591FC
